:020000040000FA
:0400000029EF06F0EE
:0400080033EF28F0BA
:04001800AAEF28F033
:1000200000EF7EF00F0B436E000EF76E420EF66E81
:100030004350F626D8B0F72AF29E0900F28EF5500A
:100040001200303132333435363738394142434487
:100050004546A2C018F019D82DC096F22EC097F2CE
:100060002FC098F230C099F231C09AF2120095C2B6
:1000700018F00BD82DC09BF22EC09CF22FC09DF221
:1000800030C09EF231C09FF212008BEC33F00AECCC
:1000900035F04AEC37F0DDEC35F04AEC37F0A0EC07
:1000A00035F05DEC31F008EC05F047EC31F031EC67
:1000B00031F0A0EF35F06951C45D02E16851C35DD4
:1000C000D8B002D0D89001D0D88012006F51C25D54
:1000D00002E16E51C15DD8B002D0D89001D0D88075
:1000E00012003AC22DF03BC22EF03CC22FF03DC2AE
:1000F00030F03EC231F0DCEC3CF02DC03FF22EC0BF
:1001000040F22FC041F230C042F231C043F24AEC1B
:1001100037F0AEEC38F005E32D6A2E6A2F6A306AAC
:10012000316A12002BC22DF02CC22EF02DC22FF0FE
:100130002EC230F02FC231F035C232F036C233F069
:1001400037C234F038C235F039C236F0DDEC35F064
:100150002DC03AF22EC03BF22FC03CF230C03DF22F
:1001600031C03EF231AE0CD0A6EC37F032C03AF2DC
:1001700033C03BF234C03CF235C03DF236C03EF2F3
:10018000120084EC33F00AEC35F017C232F018C2DA
:1001900033F019C234F01AC235F01BC236F020EC2D
:1001A00035F01CC232F01DC233F01EC234F01FC243
:1001B00035F020C236F0E3EC35F0A3B512006CC286
:1001C00032F06DC233F06EC234F06FC235F070C2DF
:1001D00036F0E3EF35F06EC018F06FC019F0D1DFE4
:1001E0002DC049F22EC04AF22FC04BF230C04CF263
:1001F00031C04DF2120074C018F075C019F0C1DFA3
:100200002DC062F22EC063F22FC064F230C065F2DE
:1002100031C066F2120061C018F062C019F0B1DF9F
:100220002DC030F22EC031F22FC032F230C033F286
:1002300031C034F212006BC018F06CC019F0A1DFAD
:100240002DC044F22EC045F22FC046F230C047F216
:1002500031C048F2120072C018F073C019F091DF7B
:100260002DC05DF22EC05EF22FC05FF230C060F292
:1002700031C061F2120068C018F069C019F081DF66
:100280002DC02BF22EC02CF22FC02DF230C02EF23A
:1002900031C02FF2120084EC33F00AEC35F021C2A9
:1002A00032F022C233F023C234F024C235F025C22A
:1002B00036F020EC35F026C232F027C233F028C2E7
:1002C00034F029C235F02AC236F0E3EC35F0A3B59C
:1002D00012006CC232F06DC233F06EC234F06FC2E5
:1002E00035F070C236F0E3EF35F070C018F071C031
:1002F00019F0D1DF2DC04EF22EC04FF22FC050F2B8
:1003000030C051F231C052F2120076C018F077C0FE
:1003100019F0C1DF2DC067F22EC068F22FC069F25C
:1003200030C06AF231C06BF212005EC018F05FC0DC
:1003300019F0B1DF2DC035F22EC036F22FC037F2E2
:1003400030C038F231C039F21200796B7B6B7C6BB4
:100350007E6B1200220E796502D0220E796F7951E0
:100360007A5DD8B403D079C07AF03D867B51795D4F
:10037000D8A00AD003C27FF07B51795DD8B404D0F5
:1003800079C07BF03D860ED07F670CD03DB808D099
:10039000806708D00A0E806F3D867B677B0702D09E
:1003A0007B6B3D861200220E7C6502D0220E7C6F94
:1003B0007C517D5DD8B405D07CC07DF03F84ADA775
:1003C0001CD07E517C5DD8A00AD003C281F07E5142
:1003D0007C5DD8B404D07CC07EF03F840ED08167B1
:1003E0000CD03DBA08D0826708D00A0E826F3F84D5
:1003F0007E677E0702D07E6B3F841200400E556EF2
:100400005C6A5D6A0FEC27F059505C265A505D22F9
:10041000552EF8D7D8905D325C32D8905D325C3280
:10042000D8905D325C3203E35C2AD8B45D2A1200B6
:10043000400E556E666B676B11EC27F059506627BE
:100440005A506723552EF8D7D89067336633D89023
:1004500067336633D8906733663303E3662BD8B4CB
:10046000672B1200080E556E666B676B5C6A5D6ADF
:10047000616B626B11EC27F0595066275A50672365
:100480000FEC27F059505C265A505D2213EC27F0F0
:10049000595061275A506223552EECD71200410E55
:1004A000366E700E356EB40E346E390E336E580ED5
:1004B000326E20D0410E366EF00E356EB40E346EB4
:1004C000390E336E580E326E15D0420E366E080E4F
:1004D000356E660E346E660E336E670E326E0AD05F
:1004E000410E366E880E356E660E346E660E336EB5
:1004F000670E326E20EC35F0B0EC32F012AE02D066
:100500000E6A0F6A1EEC31F0FF0E186E030E196EA4
:100510000F50195C02E10E50185CD8B004D018C01E
:100520000EF019C00FF012003AC22DF03BC22EF0AF
:100530003CC22FF03DC230F03EC231F0BBDF0EC0F6
:1005400098F00FC099F012003AC22DF03BC22EF085
:100550003CC22FF03DC230F03EC231F0A0DF0EC0F1
:1005600098F00FC099F012003FC22DF040C22EF05B
:1005700041C22FF042C230F043C231F03BEC37F0C1
:10058000DDEC35F09BC232F09CC233F09DC234F0FA
:100590009EC235F09FC236F020EC35F096DF0EC0DB
:1005A00098F00FC099F0120035C22DF036C22EF02F
:1005B00037C22FF038C230F039C231F071C232F098
:1005C00072C233F073C234F074C235F075C236F0C3
:1005D000DDEC35F06FDF0EC098F00FC099F012001F
:1005E00035C22DF036C22EF037C22FF038C230F0AF
:1005F00039C231F04AEC37F0E3EC35F0DFD735C2E1
:100600002DF036C22EF037C22FF038C230F039C28A
:1006100031F0D4EC3CF0E3EC35F0D0D75DC22DF0F6
:100620005EC22EF05FC22FF060C230F061C231F0C6
:1006300015D80EC092F00FC093F0120062C22DF0D8
:1006400063C22EF064C22FF065C230F066C231F092
:1006500005D80EC094F00FC095F0120071C232F0B0
:1006600072C233F073C234F074C235F075C236F022
:10067000DDEC35F01FDF12003FC22DF040C22EF03E
:1006800041C22FF042C230F043C231F03BEC37F0B0
:10069000DDEC35F096C232F097C233F098C234F0F8
:1006A00099C235F09AC236F020EC35F07BD80EC0F6
:1006B00078F012003AC22DF03BC22EF03CC22FF06F
:1006C0003DC230F03EC231F00ED03AC22DF03BC2F6
:1006D0002EF03CC22FF03DC230F03EC231F043EC70
:1006E00037F0A0EC35F05ED80EC078F0120035C2BD
:1006F0002DF036C22EF037C22FF038C230F039C29A
:1007000031F0D4EC3CF0E3EC35F019D035C22DF0EB
:1007100036C22EF037C22FF038C230F039C231F075
:100720004AEC37F0E3EC35F00AD035C22DF036C292
:100730002EF037C22FF038C230F039C231F071C21A
:1007400032F072C233F073C234F074C235F075C245
:1007500036F026D80EC078F0120030C22DF031C22B
:100760002EF032C22FF033C230F034C231F00AD052
:100770002BC22DF02CC22EF02DC22FF02EC230F045
:100780002FC231F071C232F072C233F073C234F052
:1007900074C235F075C236F003D80EC078F012007E
:1007A000DDEC35F0B0EC32F012BE0E6A1200AC6730
:1007B00002D053EC25F0010EAC6302D056EC25F0CC
:1007C000020EAC6302D059EC25F0030EAC6302D0EC
:1007D0005CEC25F0040EAC6302D05FEC25F0050E56
:1007E000AC6302D062EC25F0060EAC6302D065EC7F
:1007F00025F0070EAC6302D068EC25F0080EAC6360
:1008000002D06BEC25F0090EAC6302D06EEC25F043
:100810000A0EAC6302D071EC25F00B0EAC6302D073
:1008200074EC25F00C0EAC6302D077EC25F00D0EC5
:10083000AC6302D07AEC25F00E0EAC6302D07DECF6
:1008400025F00F0EAC6302D080EC25F0100EAC63E7
:1008500002D083EC25F0110EAC6302D086EC25F0BB
:10086000120EAC6302D089EC25F0130EAC6302D0FB
:100870008CEC25F01200AC6702D097EC25F0010E4D
:10088000AC6302D09AEC25F0020EAC6302D09DEC72
:1008900025F0030EAC6302D0A0EC25F0040EAC638F
:1008A00002D0A3EC25F0050EAC6302D0A6EC25F037
:1008B000060EAC6302D0A9EC25F0070EAC6302D0A3
:1008C000ACEC25F0080EAC6302D0AFEC25F0090EBD
:1008D000AC6302D0B2EC25F00A0EAC6302D0B5ECEA
:1008E00025F00B0EAC6302D0B8EC25F00C0EAC6317
:1008F00002D0BBEC25F00D0EAC6302D0BEEC25F0AF
:100900000E0EAC6302D0C1EC25F00F0EAC6302D02A
:10091000C4EC25F0100EAC6302D0C7EC25F0110E2C
:10092000AC6302D0CAEC25F0120EAC6302D0CDEC61
:1009300025F0130EAC6302D0D0EC25F029EC00F0CA
:10094000A3EC04F012003E9E3F900B0E9E6301D07C
:100950003E8E0C0E9E6301D03E8E100E9E6301D023
:100960003E8E110E9E6301D03E8E120E9E6301D00C
:100970003E8E0B0EA06301D03F800C0EA06301D011
:100980003F80100EA06301D03F80110EA06301D004
:100990003F80120EA06301D03F801200000E186E3F
:1009A0000CD80EC0C3F00FC0C4F0F10E186E05D8FD
:1009B0000EC0C1F00FC0C2F012006EEC33F015ECA7
:1009C00035F01CC22DF01DC22EF01EC22FF01FC22A
:1009D00030F020C231F0DDEC35F06CC232F06DC287
:1009E00033F06EC234F06FC235F070C236F0E3EC13
:1009F00035F017C232F018C233F019C234F01AC2FF
:100A000035F01BC236F0A0EC35F0317EB0EF32F09D
:100A1000410E366EF00E356E326A336A346A120059
:100A2000410E366EB00E356E326A336A346A120089
:100A3000C10E366EC80E356E326A336A346A1200E1
:100A4000000EF86E510EF76EF40EF66E43EC24F0C5
:100A500071C22DF072C22EF073C22FF074C230F04A
:100A600075C231F0D5DFE3EC35F05DEC31F09BEC95
:100A70003BF0030E376E010E386E3CEC3BF07DEC24
:100A80003AF0000EF86E510EF76EF80EF66E46EC68
:100A900024F00EC14BF10FC14CF110C14DF111C149
:100AA0004EF112C14FF1F7EC3CF06CEC3DF0E9EC8B
:100AB0003FF0000EF86E520EF76E020EF66E46EC28
:100AC00024F03EBC65EC05F01200DBEC23F0180EC0
:100AD0003DAC160E31EF24F071C276F272C277F29D
:100AE00073C278F274C279F275C27AF28D6B8E6B32
:100AF000010EB26F29EC24F0F40E8F6F010E906F8F
:100B0000000EF86E510EF76EC80EF66E43EC24F030
:100B1000000EF86E510EF76EDE0EF66E43EC24F00A
:100B2000000EF86E540EF76E480EF66E43EC24F08D
:100B300020EC05F065EC05F05B5236E0F40E8F6FAB
:100B4000010E906F3DAC3BEC37F03DBC9BEC37F0B9
:100B500071C22DF072C22EF073C22FF074C230F049
:100B600075C231F05BBE03D0E3EC35F002D0DDECB2
:100B700035F010EC05F0AEEC38F003E347EC31F063
:100B800007D018EC05F07EEC38F002E347EC31F0CA
:100B90002DC071F22EC072F22FC073F230C074F209
:100BA00031C075F25B6AC4D7906702D08F5315E0ED
:100BB000F4EC22F0C1E396EC22F0020E446206D07F
:100BC0003D7CF40E8F6F010E906FB2D70C0E446215
:100BD00001D003D0010E446228D076C218F077C24B
:100BE00019F078C21AF079C21BF07AC21CF071C2F7
:100BF0001DF072C21EF073C21FF074C220F075C2E5
:100C000021F021501C5C0BE120501B5C08E11F50BF
:100C10001A5C05E11E50195C02E11D50185CD8B445
:100C200004D021EC26F0CEEC04F0B26B5B6A446A8F
:100C300029EC24F03D821200000E31EC24F082EC0D
:100C40003BF051EC3AF001EC23F001EC23F001EF22
:100C500023F07BEC24F0D0B622D0BF2B29EC24F07B
:100C6000000EF86E5D0EF76E300EF66E43EC24F05B
:100C7000000EF86E5D0EF76E460EF66E43EC24F035
:100C80001EEC31F0BFC018F082EC3BF051EC3AF0B2
:100C900001EC23F029EC24F03D863D821ED01FECB0
:100CA00023F03EEC23F001EC23F062EC23F0BEECE9
:100CB00024F001EC23F0CFEC24F029EC24F0E6EC56
:100CC00024F03D8691893D82686B696B6A6B636B2A
:100CD000646B656B5E6A5F6A606B04005B5207E081
:100CE0005B6A09EC23F05B6A6CEC05F0F6D73DA07B
:100CF00008D0836706D0846704D03D903E9C3D9C1D
:100D00003E8632EC02F02AEC0CF0A0EC0CF065EC24
:100D10000CF03BEC01F00BEC01F095EC01F0A3B30F
:100D200023D05BEC00F020E3186A196A1A6A1B6A88
:100D30001C6A18C03FF219C040F21AC041F21BC031
:100D400042F21CC043F2A6EC37F032C03AF233C094
:100D50003BF234C03CF235C03DF236C03EF2926BFD
:100D6000936B986B996B04D092EC00F071EC00F0EF
:100D70005BEC00F000E20A0E9E6504D0E2EC07F0A6
:100D800055EC24F00A0EA06504D025EC08F067ECC1
:100D900024F06F51645D02E16E51635DD8A005D00F
:100DA00000C285F001C286F004D0856726D0866730
:100DB00024D068C06BF069C06CF063C06EF064C092
:100DC0006FF05EC070F05FC071F03AC253F23BC288
:100DD00054F23CC255F23DC256F23EC257F23FC2F7
:100DE00058F240C259F241C25AF242C25BF243C2C7
:100DF0005CF23E803E823E843E8666EC00F004E279
:100E0000E80E8D6F030E8E6F7551645D02E17451B3
:100E1000635DD8A003D002C288F002D0886712D0E8
:100E200063C074F064C075F068C072F069C073F09C
:100E30005EC076F05FC077F02BEC01F0FBEC00F0C9
:100E400085EC01F0F4EC22F01FE396EC22F0010EA9
:100E5000446204D05B6A68EC08F014D0020E44626D
:100E600004D05B6A6CEC05F00DD00B0E446204D02C
:100E70005B6A52EC09F006D00C0E446203D05B6A48
:100E80006CEC05F0446A5B6AB16705D01EEC03F0B8
:100E9000F8EC24F007D0010EB16304D00EEC03F09F
:100EA0002DEC25F0B06702D0A4EC02F0010EB06387
:100EB00002D094EC02F0020EB06302D0B4EC02F067
:100EC000030EB06302D0D4EC02F0040EB06302D083
:100ED000F0EC02F0050EB06302D0FFEC02F040EC43
:100EE00025F07BC218F07CC219F06F51195C02E149
:100EF0006E51185CD8B011D06EC07BF26FC07CF21E
:100F00006BC07DF26CC07EF270C07FF271C080F267
:100F1000AEC089F0AFC08AF012D08A6710D089675E
:100F20000ED0186A196A18C07BF219C07CF218C07A
:100F30007DF219C07EF218C07FF219C080F23DA286
:100F400005D03D923E803E823E843E86914F9189FF
:100F5000010E916300D0020E916300D0030E9163E5
:100F600005D03EA603D03E9606EC22F0040E916317
:100F700005D03EA403D03E94E8EC21F0050E916329
:100F800005D03EA203D03E92D4EC21F0060E916330
:100F900005D03EA003D03E90C0EC21F0070E916337
:100FA00000D0080E916302D075EC01F0090E916338
:100FB00002D0EBEC00F00A0E916302D01BEC01F0C2
:100FC0006DEF06F00B0E9E6305D0ADEC03F03D987F
:100FD000AD8737D00C0E9E6305D0B8EC03F03D987A
:100FE000AD872FD00D0E9E6305D065EC03F03D88D4
:100FF000AD8727D00E0E9E6305D05AEC03F03D88D6
:10100000AD871FD00F0E9E6305D03CEC03F03D88EA
:10101000AD9717D0100E9E6305D095EC03F03D9868
:10102000AD870FD0110E9E6305D086EC03F03D987E
:10103000AD8707D0120E9E6304D077EC03F03D9885
:10104000AD8778C079F0AAEF01F00B0EA06305D050
:10105000ADEC03F03D9AAD8937D00C0EA06305D0FE
:10106000B8EC03F03D9AAD892FD00D0EA06305D0EA
:1010700065EC03F03D8AAD8927D00E0EA06305D044
:101080005AEC03F03D8AAD891FD00F0EA06305D046
:101090003CEC03F03D8AAD9917D0100EA06305D04B
:1010A00095EC03F03D9AAD890FD0110EA06305D0E9
:1010B00086EC03F03D9AAD8907D0120EA06304D0F0
:1010C00077EC03F03D9AAD8978C07CF0D3EF01F066
:1010D000010EB26FDEEC23F029EC24F0000EF86E66
:1010E000540EF76EA00EF66E43EC24F0A96BA5EC3F
:1010F00008F028EC09F00DE006E2A92B030EA96523
:1011000001D0A96B05D0A907A9AF02D0030EA96F22
:10111000EED7F4EC22F012E396EC22F05B6A030EB9
:1011200044600DD0010E446203D013EC09F007D0E7
:10113000020E446203D013EC09F001D0DAD729EC97
:1011400024F03D82B26B446A1200DEEC23F0A96702
:1011500018D0000EF86E540EF76EB60EF66E43EC15
:1011600024F0000EF86E540EF76ECC0EF66E43ECC3
:1011700024F0000EF86E540EF76EE20EF66E43EC9D
:1011800024F0010EA96318D0000EF86E550EF76E0C
:10119000240EF66E43EC24F0000EF86E550EF76E3A
:1011A0003A0EF66E43EC24F0000EF86E550EF76E14
:1011B000500EF66E43EC24F0020EA96318D0000E18
:1011C000F86E550EF76E660EF66E43EC24F0000EC8
:1011D000F86E550EF76E7C0EF66E43EC24F0000EA2
:1011E000F86E550EF76E920EF66E43EC24F0030E79
:1011F000A96318D0000EF86E550EF76EBE0EF66E8F
:1012000043EC24F0000EF86E550EF76ED40EF66E19
:1012100043EC24F0000EF86E550EF76EEA0EF66EF3
:1012200043EC24F01200A96702D0B4EF1DF0010EC8
:10123000A96302D0B5EF1EF0020EA96302D056EFEB
:101240001FF0030EA96302D0B8EF1FF029EF24F0BE
:101250005B5211E05BAE08D05B50E86CFE0B0BE01C
:101260005B6AD894D88008D05B50FE0B04E05B6AC0
:10127000D894D89001D0D88412005B5211E05BAEB4
:1012800008D05B50E86CFF0B0BE05B6AD894D88009
:1012900008D05B50FF0B04E05B6AD894D89001D073
:1012A000D88412003E88010EB26F29EC24F0000EA3
:1012B000F86E570EF76E340EF66E43EC24F090EC99
:1012C00009F028EC09F00DE006E2AA2B140EAA653D
:1012D00001D0AA6B05D0AA07AAAF02D0140EAA6F3C
:1012E000EED7F4EC22F013E396EC22F0030E446008
:1012F0000FD0010E446204D05B6ABDEC0BF008D045
:10130000020E446204D05B6ABDEC0BF001D0D9D769
:1013100029EC24F05B6A3D82B26B446A3E9812006D
:10132000DEEC23F0AA670CD0000EF86E570EF76EB5
:101330004A0EF66E43EC24F0B7EC28F0B5EC28F03A
:10134000010EAA6318D0000EF86E570EF76E600EED
:10135000F66E43EC24F0000EF86E570EF76E760E24
:10136000F66E43EC24F0000EF86E570EF76E8C0EFE
:10137000F66E43EC24F0020EAA6318D0000EF86E4D
:10138000570EF76EA20EF66E43EC24F0000EF86EC8
:10139000570EF76EB80EF66E43EC24F0000EF86EA2
:1013A000570EF76ECE0EF66E43EC24F0030EAA63D2
:1013B00018D0000EF86E570EF76EE40EF66E43EC82
:1013C00024F0000EF86E570EF76EFA0EF66E43EC30
:1013D00024F0000EF86E580EF76E100EF66E43EC09
:1013E00024F0040EAA6318D0000EF86E580EF76EA3
:1013F0005C0EF66E43EC24F0000EF86E580EF76E9D
:10140000720EF66E43EC24F0000EF86E580EF76E76
:10141000880EF66E43EC24F0050EAA6318D0000E79
:10142000F86E580EF76EB40EF66E43EC24F0000E14
:10143000F86E580EF76ECA0EF66E43EC24F0000EEE
:10144000F86E580EF76EE00EF66E43EC24F0060EC2
:10145000AA6318D0000EF86E590EF76E0C0EF66ED9
:1014600043EC24F0000EF86E590EF76E220EF66E65
:1014700043EC24F0000EF86E590EF76E380EF66E3F
:1014800043EC24F0070EAA6318D0000EF86E590E34
:10149000F76E4E0EF66E43EC24F0000EF86E590E09
:1014A000F76E220EF66E43EC24F0000EF86E590E25
:1014B000F76E380EF66E43EC24F0080EAA6318D0CF
:1014C000000EF86E590EF76E640EF66E43EC24F0C3
:1014D000000EF86E590EF76E7A0EF66E43EC24F09D
:1014E000000EF86E590EF76E900EF66E43EC24F077
:1014F000090EAA6318D0000EF86E590EF76ECA0EC8
:10150000F66E43EC24F0000EF86E590EF76EE00E06
:10151000F66E43EC24F0000EF86E590EF76EF60EE0
:10152000F66E43EC24F00A0EAA6318D0000EF86E93
:101530005A0EF76E340EF66E43EC24F0000EF86E81
:101540005A0EF76E4A0EF66E43EC24F0000EF86E5B
:101550005A0EF76E600EF66E43EC24F00B0EAA6383
:1015600018D0000EF86E5A0EF76EAA0EF66E43EC07
:1015700024F0000EF86E5A0EF76EC00EF66E43ECB5
:1015800024F0000EF86E5A0EF76ED60EF66E43EC8F
:1015900024F00C0EAA6318D0000EF86E5A0EF76EE7
:1015A000EC0EF66E43EC24F0000EF86E5A0EF76E59
:1015B000C00EF66E43EC24F0000EF86E5A0EF76E75
:1015C000D60EF66E43EC24F00D0EAA6318D0000E72
:1015D000F86E5B0EF76E020EF66E43EC24F0000E12
:1015E000F86E5B0EF76E180EF66E43EC24F0000EEC
:1015F000F86E5B0EF76E2E0EF66E43EC24F00E0EB8
:10160000AA6318D0000EF86E5B0EF76E780EF66EB9
:1016100043EC24F0000EF86E5B0EF76E8E0EF66E45
:1016200043EC24F0000EF86E5B0EF76EA40EF66E1F
:1016300043EC24F00F0EAA6318D0000EF86E5C0E77
:10164000F76E960EF66E43EC24F0000EF86E5C0E0C
:10165000F76EAC0EF66E43EC24F0000EF86E5C0EE6
:10166000F76EC20EF66E43EC24F0100EAA6318D08B
:10167000000EF86E5C0EF76EEE0EF66E43EC24F084
:10168000000EF86E5D0EF76E040EF66E43EC24F05D
:10169000000EF86E5D0EF76E1A0EF66E43EC24F037
:1016A000110EAA6318D0000EF86E5D0EF76E520E82
:1016B000F66E43EC24F0000EF86E5D0EF76E680EC9
:1016C000F66E43EC24F0000EF86E5D0EF76E7E0EA3
:1016D000F66E43EC24F0120EAA6318D0000EF86EDA
:1016E0005D0EF76EC20EF66E43EC24F0000EF86E3F
:1016F0005D0EF76ED80EF66E43EC24F0000EF86E19
:101700005D0EF76EEE0EF66E43EC24F0130EAA6338
:1017100018D0000EF86E5E0EF76E040EF66E43ECF7
:1017200024F0000EF86E5E0EF76E1A0EF66E43ECA5
:1017300024F0000EF86E5E0EF76E300EF66E43EC7F
:1017400024F0140EAA6318D0000EF86E5F0EF76E28
:10175000A60EF66E43EC24F0000EF86E5F0EF76EE8
:10176000BC0EF66E43EC24F0000EF86E5F0EF76EC2
:10177000D20EF66E43EC24F0120029EC24F0AA6796
:1017800001D064D0010EAA6302D033EF0EF0020E36
:10179000AA6302D004EF0FF0030EAA6302D059EF40
:1017A00011F0040EAA6302D0ADEF12F0050EAA6389
:1017B00002D065EF13F0060EAA6302D0DCEF13F03F
:1017C000070EAA6302D02EEF14F0080EAA6302D00F
:1017D00080EF14F0090EAA6302D041EF15F00A0E53
:1017E000AA6302D09BEF15F00B0EAA6302D07EEF26
:1017F0000DF00C0EAA6302D0B0EF0DF00D0EAA632F
:1018000002D04FEF16F00E0EAA6302D0F1EF16F0E1
:101810000F0EAA6302D0FBEF17F0100EAA6302D0DE
:1018200061EF18F0110EAA6302D099EF18F0120EB2
:10183000AA6302D092EF19F0130EAA6302D005EF4B
:101840001AF0140EAA6302D045EF1DF029EC24F023
:101850003D821200A3A933D0D890683769376A3720
:10186000D890683769376A37D890683769376A37E8
:1018700010EC31F066C018F067C019F018506827F6
:10188000195069231A506A231EEC31F068C018F011
:1018900069C019F06AC01AF0090E1D6E86EC39F0A5
:1018A00018C068F019C069F01AC06AF0040E1D640F
:1018B00005D0682BD8B4692BD8B46A2B05D06A6BD5
:1018C00066C068F067C069F01200A3A733D0D89053
:1018D000633764376537D890633764376537D89096
:1018E00063376437653710EC31F061C018F062C0BF
:1018F00019F018506327195064231A5065231EEC01
:1019000031F063C018F064C019F065C01AF0090E18
:101910001D6E86EC39F018C063F019C064F01AC06F
:1019200065F0040E1D6405D0632BD8B4642BD8B4C5
:10193000652B05D0656B61C063F062C064F0120076
:10194000A3AB33D0D8905E365F366037D8905E3622
:101950005F366037D8905E365F36603710EC31F016
:101960005CC018F05DC019F018505E2619505F2257
:101970001A5060231EEC31F05EC018F05FC019F001
:1019800060C01AF0090E1D6E86EC39F018C05EF0CA
:1019900019C05FF01AC060F0040E1D6405D05E2A05
:1019A000D8B45F2AD8B4602B05D0606B5CC05EF001
:1019B0005DC05FF01200530E31EC24F0200E3DAEFE
:1019C0003C0E8BEC23F0270E31EC24F0200E3DBEB4
:1019D0003C0E8BEC23F01200000EF86E520EF76EE8
:1019E0008E0EF66E43EC24F01EEC31F015C218F0AA
:1019F00016C219F082EC3BF051EC3AF0DBEC23F02C
:101A0000B36702D0490E09D0010EB36302D0480E6D
:101A100004D0020EB36301D0470E31EC24F0120063
:101A2000B36B010EB26F3DBE09D0000EF86E520EC0
:101A3000F76E4A0EF66E43EC24F008D0000EF86EF6
:101A4000520EF76E600EF66E43EC24F0000EF86E48
:101A5000540EF76E740EF66E43EC24F0000EF86E22
:101A6000520EF76E960EF66E43EC24F0ECEC0CF092
:101A70005B522BE015C218F016C219F0B36705D0FF
:101A8000010E1D6E000E1E6E0FD0010EB36305D049
:101A90000A0E1D6E000E1E6E07D0020EB36304D038
:101AA000640E1D6E000E1E6E5BBE05D01D50182606
:101AB0001E50192204D01D50185E1E50195A18C00D
:101AC00015F219C016F25B6AAED7F4EC22F0D0E33F
:101AD00096EC22F0020E446206D0B32B030EB363E1
:101AE00001D0B36BA0D70B0E446202D0D88005D0D2
:101AF000010E446202D0D89000D01200E1EC0DF04B
:101B00001CC22DF01DC22EF01EC22FF01FC230F0DD
:101B100020C231F017C232F018C233F019C234F0CB
:101B20001AC235F01BC236F0B9EC13F015C245F0FD
:101B300016C246F013C215F214C216F229EC24F0B4
:101B40003D9E6EDF0CE23D8E15C213F216C214F2FA
:101B500045C015F246C016F263DF01E2D6D012008E
:101B6000E1EC0DF026C22DF027C22EF028C22FF096
:101B700029C230F02AC231F021C232F022C233F041
:101B800023C234F024C235F025C236F0B9EC13F08C
:101B900015C245F016C246F013C215F214C216F271
:101BA00029EC24F03D9E3CDFDAE23D8E15C213F2B3
:101BB00016C214F245C015F246C016F231DFCFE26C
:101BC00075D117C281F218C282F219C283F21AC209
:101BD00084F21BC285F21CC286F21DC287F21EC2AD
:101BE00088F21FC289F220C28AF221C28BF222C27D
:101BF0008CF223C28DF224C28EF225C28FF226C24D
:101C000090F227C291F228C292F229C293F22AC21C
:101C100094F2120081C217F282C218F283C219F242
:101C200084C21AF285C21BF286C21CF287C21DF260
:101C300088C21EF289C21FF28AC220F28BC221F230
:101C40008CC222F28DC223F28EC224F28FC225F200
:101C500090C226F291C227F292C228F293C229F2D0
:101C600094C22AF21200E1EC0DF0A3C045F0A38962
:101C7000DEEC23F029EC24F0000EF86E530EF76E24
:101C8000E40EF66E43EC24F0000EF86E540EF76E80
:101C9000480EF66E43EC24F0686B696B6A6B94D95E
:101CA000F4EC22F0FCE396EC22F0010E446286D0C4
:101CB00068C013F269C014F229EC24F0000EF86E2B
:101CC000530EF76EFA0EF66E43EC24F0000EF86E2B
:101CD000540EF76E480EF66E43EC24F0686B696B99
:101CE0006A6B72D9F4EC22F0FCE396EC22F0010E60
:101CF000446264D068C015F269C016F264D8FFEC83
:101D000022F0FFEC22F045C0A3F029EC24F0000EF5
:101D1000F86E540EF76E100EF66E43EC24F02DD9CB
:101D20002DC017F22EC018F22FC019F230C01AF2CF
:101D300031C01BF243D92DC01CF22EC01DF22FC0A2
:101D40001EF230C01FF231C020F280D9FFEC22F029
:101D5000000EF86E540EF76E740EF66E43EC24F01F
:101D600096EC22F0010E446229D029EC24F099D996
:101D7000FFEC22F0000EF86E540EF76E740EF66E45
:101D800043EC24F096EC22F0010E446217D029ECCB
:101D900024F042DAFFEC22F0000EF86E540EF76EDB
:101DA000740EF66E43EC24F096EC22F0010E4462C1
:101DB00005D043EC26F0CEEC04F004D00AEC0EF093
:101DC0003AEC1FF01200000EF86E600EF76E6C0E0B
:101DD000F66E43EC24F0000EF86E600EF76E820E85
:101DE000F66E43EC24F0000EF86E600EF76E980E5F
:101DF000F66E43EC24F0000EF86E600EF76EAE0E39
:101E0000F66E43EC24F01200E1EC0DF0A3C045F0B7
:101E1000A38BDEEC23F029EC24F0000EF86E530EB9
:101E2000F76EE40EF66E43EC24F0000EF86E540EDE
:101E3000F76E480EF66E43EC24F05E6A5F6A606BE4
:101E4000E4D8F4EC22F0FCE396EC22F0010E4462BC
:101E500084D05EC013F25FC014F229EC24F0000EAF
:101E6000F86E530EF76EFA0EF66E43EC24F0000E89
:101E7000F86E540EF76E480EF66E43EC24F05E6A70
:101E80005F6A606BC2D8F4EC22F0FCE396EC22F0BF
:101E9000010E446262D05EC015F25FC016F293DF9D
:101EA000FFEC22F0FFEC22F045C0A3F029EC24F077
:101EB000000EF86E540EF76E260EF66E43EC24F00C
:101EC0005CD82DC021F22EC022F22FC023F230C0E8
:101ED00024F231C025F272D82DC026F22EC027F28E
:101EE0002FC028F230C029F231C02AF2AFD8FFEC5F
:101EF00022F0000EF86E540EF76E740EF66E43EC80
:101F000024F096EC22F0010E446227D029EC24F054
:101F1000FFD8FFEC22F0000EF86E540EF76E740E30
:101F2000F66E43EC24F096EC22F0010E446215D0DC
:101F300029EC24F024D9FFEC22F0000EF86E540EA8
:101F4000F76E740EF66E43EC24F096EC22F0010E60
:101F5000446203D055EC26F004D00AEC0EF03AECC3
:101F60001FF01200000E31EC24F0E5EC3BF00EEC1B
:101F70003CF0FFEC22F096EF22F013C218F014C2EE
:101F800019F084EC33F00AEC35F0E1EC31F015C2D5
:101F900018F016C219F084EC33F015EC35F0DDECD6
:101FA00035F05DEC31F01E0E186E8BEC33F00AEC60
:101FB00035F031EC31F0A0EC35F0120073EC31F07B
:101FC00020EC35F0317E1200DEEC23F00BEC23F038
:101FD00018EC02F02AEC0CF0000EF86E530EF76EBF
:101FE000C00EF66E43EC24F068C018F069C019F01A
:101FF00084EC33F00AEC35F09BEC3BF0050E376EC9
:10200000386A3CEC3BF07DEF3AF0DEEC23F00BEC71
:1020100023F0FEEC01F0A0EC0CF0000EF86E530E75
:10202000F76ED80EF66E43EC24F05EC018F05FC079
:1020300019F084EC33F00AEC35F09BEC3BF0050E24
:10204000376E386A3CEC3BF07DEF3AF0DEEC23F083
:10205000000EF86E520EF76E760EF66E43EC24F01C
:102060001EEC31F013C218F014C219F082EC3BF0F0
:10207000040E376E51EC3AF0000EF86E520EF76E09
:10208000820EF66E43EC24F01EEC31F015C218F00F
:1020900016C219F082EC3BF0040E376E51EC3AF0A8
:1020A0001200DEEC23F0000EF86E540EF76E100EE8
:1020B000F66E43EC24F0000EF86E540EF76E3C0EF4
:1020C000F66E43EC24F017C22DF018C22EF019C2A0
:1020D0002FF01AC230F01BC231F0E5EC3BF00EECF1
:1020E0003CF0000EF86E540EF76E420EF66E43ECA6
:1020F00024F01CC22DF01DC22EF01EC22FF01FC2F4
:1021000030F020C231F0E5EC3BF00EEC3CF0120078
:10211000DEEC23F0000EF86E540EF76E260EF66E0F
:1021200043EC24F0000EF86E540EF76E3C0EF66E83
:1021300043EC24F021C22DF022C22EF023C22FF056
:1021400024C230F025C231F0E5EC3BF00EEC3CF05F
:10215000000EF86E540EF76E420EF66E43EC24F04D
:1021600026C22DF027C22EF028C22FF029C230F04F
:102170002AC231F0E5EC3BF00EEC3CF01200DEEC54
:1021800023F0000EF86E540EF76E260EF66E43EC3A
:1021900024F0000EF86E540EF76E3C0EF66E43EC13
:1021A00024F021C218F022C219F023C21AF024C26E
:1021B0001BF025C21CF01C503AEC24F01B503AECEA
:1021C00024F01A503AEC24F019503AEC24F018504C
:1021D0003AEC24F0000EF86E540EF76E420EF66ED6
:1021E00043EC24F026C218F027C219F028C21AF0D6
:1021F00029C21BF02AC21CF01C503AEC24F01B50E0
:102200003AEC24F01A503AEC24F019503AEC24F04D
:1022100018503AEC24F01200DEEC23F0000EF86EB9
:10222000540EF76E100EF66E43EC24F0000EF86EAE
:10223000540EF76E3C0EF66E43EC24F017C218F005
:1022400018C219F019C21AF01AC21BF01BC21CF0F6
:102250001C503AEC24F01B503AEC24F01A503AECA3
:1022600024F019503AEC24F018503AEC24F0000E07
:10227000F86E540EF76E420EF66E43EC24F01CC25C
:1022800018F01DC219F01EC21AF01FC21BF020C2A6
:102290001CF01C503AEC24F01B503AEC24F01A507D
:1022A0003AEC24F019503AEC24F018503AEC24F0AF
:1022B0001200DEEC23F0B36B29EC24F0000EF86E74
:1022C000580EF76E260EF66E43EC24F0000EF86EF4
:1022D000580EF76E3C0EF66E43EC24F0000EF86ECE
:1022E000540EF76E480EF66E43EC24F06CC22DF0DF
:1022F0006DC22EF06EC22FF06FC230F070C231F09E
:102300006CC24AF06DC24BF06EC24CF06FC24DF021
:1023100070C24EF0D4EC3CF0A0EC35F0DDEC36F0C1
:10232000DDEC37F0A1EC32F0EFEC37F02DC045F0EA
:102330002EC046F02FC047F030C048F031C049F001
:102340005B6ADBEC23F0000EF86E580EF76E520E4F
:10235000F66E43EC24F045C02DF046C02EF047C089
:102360002FF048C030F049C031F09BEC3BF0030E39
:10237000376E010E386E3CEC3BF07DEC3AF0000E0F
:10238000F86E580EF76E580EF66E43EC24F045C00A
:102390002DF046C02EF047C02FF048C030F049C0A5
:1023A00031F060EC38F0D4EC3CF020EC35F09BECF4
:1023B0003BF0050E376E030E386E3CEC3BF07DECC7
:1023C0003AF0000EF86E620EF76E180EF66E46ECDE
:1023D00024F0B36702D01B0E04D0010EB36301D00A
:1023E000190E31EC24F0B36702D09BEC37F0010EEC
:1023F000B36302D03BEC37F03DEC09F02BE00DE28B
:1024000045C02DF046C02EF047C02FF048C030F038
:1024100049C031F0E3EC35F011D045C02DF046C095
:102420002EF047C02FF048C030F049C031F0DDEC4D
:1024300035F03BEC37F002E347EC31F02DC045F0CE
:102440002EC046F02FC047F030C048F031C049F0F0
:102450005B6A79D7F4EC22F0C6E396EC22F0010E29
:1024600044621DD045C02DF046C02EF047C02FF06D
:1024700048C030F049C031F060EC38F0D4EC3CF0AA
:1024800020EC35F02DC06CF22EC06DF22FC06EF234
:1024900030C06FF231C070F267EC26F016D0020E39
:1024A000446206D0B32B020EB3634DD7B36B4BD748
:1024B000020E446448D74AC06CF24BC06DF24CC067
:1024C0006EF24DC06FF23AEC1FF012000AEC35F0DC
:1024D000F2EC37F0420E366E700E356E326A336AA9
:1024E000346AA0EC35F09BEC3BF0030E376E010E26
:1024F000386E3CEC3BF07DEC3AF0000EF86E610E6D
:10250000F76E540EF66E46EC24F012000AEC35F02D
:10251000F2EC37F09BEC3BF0040E376E020E386E97
:102520000AD00AEC35F0F2EC37F09BEC3BF0040EED
:10253000376E010E386E3CEC3BF07DEC3AF0000E4D
:10254000F86E610EF76E500EF66E46EC24F0120037
:10255000200E31EC24F0DBEF23F000C245F001C285
:1025600046F0DEEC23F0000EF86E580EF76E9E0E6D
:10257000F66E43EC24F0000EF86E600EF76EC40E9B
:10258000F66E43EC24F0000EF86E540EF76E480E13
:10259000F66E43EC24F0000EF86E600EF76EDA0E65
:1025A000F66E43EC24F000C218F001C219F084EC7E
:1025B00033F0B7DFCDDF3DEC09F03EE01CE200C2B6
:1025C00018F001C219F00A0E1D6E000E1E6E1D508D
:1025D00018261E501922E80E1D6E030E1E6E19508D
:1025E0001E5C02E118501D5CD8B004D01DC018F06C
:1025F0001EC019F01BD000C218F001C219F00A0E5B
:102600001D6E000E1E6E1D50185E1E50195A320EA1
:102610001D6E000E1E6E19501E5C02E118501D5CEE
:10262000D8A004D01DC018F01EC019F018C000F2C8
:1026300019C001F25B6A95D7F4EC22F0BCE396EC8A
:1026400022F0DEEC23F0030E446006D0010E44625B
:1026500003D08BEC26F006D045C000F246C001F254
:102660003AEC1FF012004E0E31EC24F0DBEF23F0B9
:10267000196A1A6A1B6A1C6A25EC31F0050E1D6E78
:1026800086EC39F01806186602D0010E186E25EC9B
:1026900031F0050E1D6E12EC39F01200196A1A6A3B
:1026A0001B6A1C6A25EC31F0050E1D6E86EC39F0B4
:1026B000182A25EC31F0050E1D6E12EC39F0FA0ED9
:1026C000186402D0FA0E186E1200010EB26F3D9E11
:1026D00003C245F0DEEC23F0000EF86E580EF76EE4
:1026E000F60EF66E43EC24F0000EF86E540EF76E04
:1026F000480EF66E43EC24F0000EF86E610EF76E95
:102700003E0EF66E43EC24F003C218F08BEC33F06F
:10271000FDDEA9DF3DEC09F00DE005E203C218F093
:102720004EEC13F004D003C218F038EC13F018C0CC
:1027300003F2D0D7F4EC22F0EDE3DEEC23F096ECDC
:1027400022F0010E446203D09DEC26F011D0020E5F
:10275000446201D0F9D70B0E446201D003D00C0EB5
:10276000446206D045C003F246C004F23AEC1FF0C2
:1027700012005DEC31F0D6EC31F0A0EC35F0317E9A
:10278000B0EC32F00EC013F20FC014F23CEC31F09A
:102790001E0E186E8BEC33F015EC35F0E3EC35F0D3
:1027A00073EC31F0A0EC35F0317EB0EC32F00EC0BD
:1027B00015F20FC016F21200DEEC23F01CC22DF051
:1027C0001DC22EF01EC22FF01FC230F020C231F009
:1027D00017C232F018C233F019C234F01AC235F001
:1027E0001BC236F0C6DF29EC24F0000EF86E540E42
:1027F000F76E100EF66E43EC24F026EC10F0FFECB2
:1028000022F0000EF86E540EF76E740EF66E43EC66
:1028100024F096EC22F029EC24F051EC10F0FFECBF
:1028200022F0000EF86E540EF76E740EF66E43EC46
:1028300024F096EC22F029EC24F00CEC11F0FFECE3
:1028400022F0000EF86E540EF76E740EF66E43EC26
:1028500024F096EC22F029EC24F01200DEEC23F0B8
:1028600026C22DF027C22EF028C22FF029C230F048
:102870002AC231F021C232F022C233F023C234F036
:1028800024C235F025C236F074DF29EC24F0000EA6
:10289000F86E540EF76E260EF66E43EC24F026EC1E
:1028A00010F0FFEC22F0000EF86E540EF76E740E6E
:1028B000F66E43EC24F096EC22F029EC24F088EC40
:1028C00010F0FFEC22F0000EF86E540EF76E740E4E
:1028D000F66E43EC24F096EC22F029EC24F0BFECE9
:1028E00010F0FFEC22F0000EF86E540EF76E740E2E
:1028F000F66E43EC24F096EC22F029EC24F0120062
:10290000DEEC23F029EC24F0000EF86E590EF76E81
:10291000A60EF66E43EC24F0796B7C6B7B6B7E6BC2
:102920003D983D8A79EC24F0926B936B2DEC25F069
:10293000986B996B40EC25F0FF0E186E030E196E24
:1029400084EC33F00AEC35F0220E186E8BEC33F089
:1029500015EC35F0A0EC35F05DEC31F0000EF86EC2
:10296000520EF76E360EF66E43EC24F0000EF86E43
:10297000520EF76E3C0EF66E43EC24F0000EF86E2D
:10298000590EF76EBC0EF66E43EC24F01EEC31F0DF
:1029900079C018F082EC3BF0020E376E51EC3AF041
:1029A000000EF86E590EF76EC40EF66E43EC24F06E
:1029B0001EEC31F098C018F099C019F082EC3BF091
:1029C000040E376E51EC3AF03DEC09F030E00AE2CB
:1029D000792B7C2B220E796504D0220E796F220E82
:1029E0007C6F06D079077C0779AF02D0796B7C6B5E
:1029F0007CC07EF03D983D8A79EC24F079C018F0D7
:102A00008BEC33F00AEC35F031EC31F020EC35F0A2
:102A1000B0EC32F00EC092F00FC093F02DEC25F028
:102A20000EC098F00FC099F040EC25F0A7D7F4EC59
:102A300022F0CAE396EC22F0030E446008D0010EA7
:102A4000446201D005D0020E446201D001D096D775
:102A500029EC24F0796B7C6B3D983D8A79EC24F06D
:102A6000926B936B2DEC25F0986B996B40EC25F0F5
:102A70003D8212004F0E3DBE230E31EC24F0DBEF01
:102A800023F0DEEC23F029EC24F03D9EADC045F0B0
:102A9000DEEC23F0020EB26F000EF86E5A0EF76EE7
:102AA0000C0EF66E43EC24F0000EF86E540EF76E2A
:102AB000480EF66E43EC24F0000EF86E5A0EF76ED8
:102AC000220EF66E43EC24F0780EADA1200E8BECB6
:102AD00023F0000EF86E520EF76EAC0EF66E46EC5A
:102AE00024F05B5203E0AD715B6AD2D7F4EC22F0C4
:102AF000F8E3DEEC23F096EC22F0010E446203D002
:102B0000AFEC26F00DD0020E446200D00B0E4462F2
:102B100000D00C0E446200D045C0ADF03AEC1FF07E
:102B200029EC24F03D8212004D0E3DBE230E31EC07
:102B300024F0DBEF23F0DEEC23F029EC24F0ADC031
:102B400045F03D9E020EB26FDEEC23F0000EF86EF3
:102B50005A0EF76E760EF66E43EC24F0000EF86E09
:102B6000540EF76E5E0EF66E43EC24F0000EF86E17
:102B70005A0EF76E8C0EF66E43EC24F0AEC018F0D1
:102B8000AFC019F084EC33F066EC12F0000EF86E72
:102B90005A0EF76E980EF66E43EC24F0780EADA543
:102BA000200E8BEC23F0000EF86E520EF76EAC0E7A
:102BB000F66E46EC24F0DBEC0CF0B6DFAEC018F09D
:102BC000AFC019F0B80E1D6E0B0E1E6E3DEC09F075
:102BD00035E016E23DBE2FD01D5018261E5019229A
:102BE000600E1D6EEA0E1E6E19501E5C02E118503A
:102BF0001D5CD8B004D01DC018F01EC019F015D04F
:102C00003DBE13D01D50185E1E50195A700E1D6E19
:102C1000170E1E6E1E50195C02E11D50185CD8B0D4
:102C200004D01DC018F01EC019F018C0AEF019C0B5
:102C3000AFF05B6A87D7AD755B6A84D7F4EC22F09E
:102C4000BDE3DEEC23F096EC22F0010E446209D0E5
:102C5000AFEC26F0D9EC25F0AEC089F0AFC08AF019
:102C600011D0020E446202D03D7E6CD70B0E44623E
:102C700002D03D7E67D70C0E446200D045C0ADF057
:102C80003AEC1FF01200210E06D0230E04D04B0E9A
:102C900002D0260E00D031EC24F0DBEF23F0DEEC86
:102CA00023F029EC24F002C245F0ADC046F03D9E71
:102CB000020EB26FDEEC23F0000EF86E5B0EF76EC4
:102CC000440EF66E43EC24F0000EF86E540EF76ED0
:102CD0005E0EF66E43EC24F0000EF86E5B0EF76E9F
:102CE0005A0EF66E43EC24F002C218F08BEC33F06F
:102CF00086EC12F0000EF86E5B0EF76E640EF66E48
:102D000043EC24F0780EADA3200E8BEC23F0000EE4
:102D1000F86E520EF76EAC0EF66E46EC24F03DAE39
:102D2000B6DF3DBEB6DF3DEC09F01DE00EE23DAE84
:102D300003D0AD735B6ABCD702C218F0182AFA0E32
:102D4000186402D0FA0E186E0AD03DAE03D0AD73EF
:102D50005B6AAED702C218F0180618BE186A18C00F
:102D600002F25B6AA5D7F4EC22F0DDE3DEEC23F09F
:102D700096EC22F0010E446205D0AFEC26F079EC1F
:102D800026F013D0020E446202D03D7E91D70B0E86
:102D9000446202D03D7E8CD70C0E446200D045C008
:102DA00002F246C0ADF03AEC1FF01200000EF86ED1
:102DB000600EF76EEE0EF66E43EC24F08BEC33F003
:102DC0000AEC35F04AEC37F0A0EC35F09BEC3BF028
:102DD000030E376E010E386E3CEC3BF07DEC3AF0A2
:102DE0001200000EF86EFC0EF76E000EF66E090073
:102DF000F550186E040E186273D00900F550186E65
:102E0000000E18626DD00900F550186EF00E1862B1
:102E100067D00900F550186E0E0E186261D0EBEC09
:102E200017F0000EF86E5B0EF76EBA0EF66E43ECFE
:102E300024F0000EF86E5B0EF76ED00EF66E43ECCB
:102E400024F0000EF86E5B0EF76EE60EF66E43ECA5
:102E500024F0000EF86E540EF76E8A0EF66E43ECF8
:102E600024F0F4EC22F037E2F3EC17F0FAE2186EFB
:102E7000400E1862F6D793EC17F0F4EC22F02BE238
:102E8000F3EC17F0FAE2186E3B0E186201D00DD089
:102E900000EE46F04550E92618C0EFFF452A090E1E
:102EA0004562EBD793EC17F0DCD7760E466206D07E
:102EB000010E456203D0BFEC17F009D0670E4662E1
:102EC00006D0060E456203D09BEC17F000D093ECC1
:102ED00017F031EF17F096EC22F03AEC1FF01200E9
:102EE000000EF86E5B0EF76EFC0EF66E43EC24F0EF
:102EF000000EF86E5C0EF76E120EF66E43EC24F0C8
:102F0000000EF86E5C0EF76E280EF66E43EC24F0A1
:102F1000000EF86E5C0EF76E3E0EF66E43EC24F07B
:102F2000FFEC22F012000A0E546E00EE45F0EE6A3D
:102F3000542EFDD71200230E476220D0230E486284
:102F40001DD0230E49621AD0230E4A6217D0230ED9
:102F50004B6214D0000EF86E5C0EF76E6A0EF66EC1
:102F600043EC24F0000EF86E5C0EF76E800EF66EE9
:102F700043EC24F001EC23F010EF00F01200000EFF
:102F8000F86E5C0EF76E540EF66E43EC24F0B7EC60
:102F900028F0400EE6EC17F0760EE6EC17F0510E36
:102FA000E6EC17F0570EE6EC17F01EEC31F06E0E63
:102FB000186E82EC3BF0030E376E386A010E3C6EE1
:102FC00051EC3AF03B0EE6EC17F0120004009EA81C
:102FD000FDD7AD6E12000400440EAF6EAC84AC8A17
:102FE000AB88AB8E120004009EAA03D0AE50D890DE
:102FF0001200D880120029EC24F095C245F0DEECD6
:1030000023F0000EF86E5C0EF76ED80EF66E43ECF1
:1030100024F0000EF86E610EF76E120EF66E43ECA1
:1030200024F0000EF86E540EF76E480EF66E43EC68
:1030300024F095C218F0D6EC16F045EC16F028EC0A
:1030400009F016E095C218F003E2050E182602D02A
:10305000050E185E0F0E186002D00F0E186E640E6B
:10306000186402D0640E186E18C095F25B6AC7D758
:10307000F4EC22F0E4E3DEEC23F096EC22F0030E15
:10308000446006D0010E446203D0C1EC26F016D095
:1030900045C09BF246C09CF247C09DF248C09EF2DC
:1030A00049C09FF229EC24F0000EF86E530EF76E23
:1030B000A80EF66E43EC24F0FFEC22F037EC00F0A3
:1030C000120029EC24F0DEEC23F0000EF86E5D0E09
:1030D000F76E300EF66E43EC24F0000EF86E540ED0
:1030E000F76E740EF66E43EC24F0000EF86E5D0E73
:1030F000F76E460EF66E43EC24F01EEC31F0BFC0C6
:1031000018F082EC3BF051EC3AF096EC22F0120011
:10311000466603D00D0EC06F0BD0010E466203D081
:103120000E0EC06F05D0020E466202D00F0EC06FA9
:103130001200C0C045F029EC24F0DEEC23F0000EB4
:10314000F86E5D0EF76E940EF66E43EC24F0000EF2
:10315000F86E540EF76E480EF66E43EC24F0D8DF8E
:10316000DEEC23F0000EF86E5D0EF76EAA0EF66E22
:1031700043EC24F0000EF86E5D0EF76EB80EF66E9E
:1031800043EC24F0DBEC23F028EC09F00DE006E240
:10319000462A030E466207D0466A05D0460646AE6A
:1031A00002D0020E466EDBD7F4EC22F0EDE3DEEC4B
:1031B00023F096EC22F0030E446006D0010E446228
:1031C00003D00FEC26F00ED045C0C0F029EC24F05F
:1031D000000EF86E530EF76EA80EF66E43EC24F058
:1031E000FFEC22F0120029EC24F0D5EC19F0000ECF
:1031F000F86E520EF76ECA0EF66E43EC24F0780E9F
:10320000A3B1200E8BEC23F0000EF86E520EF76E79
:10321000AC0EF66E46EC24F0000EF86E520EF76E11
:10322000DA0EF66E43EC24F0780EA3B3200E8BEC8E
:1032300023F0000EF86E520EF76EAC0EF66E46ECF2
:1032400024F0120029EC24F0000EF86E520EF76EF6
:10325000EA0EF66E43EC24F0780EA3B5200E8BEC4C
:1032600023F0000EF86E520EF76EAC0EF66E46ECC2
:1032700024F0000EF86E520EF76EFA0EF66E43EC66
:1032800024F0A2C018F0DEEC16F0000EF86E520E1C
:10329000F76EAC0EF66E46EC24F0B7EC28F0120098
:1032A00029EC24F0000EF86E530EF76E0A0EF66E3F
:1032B00043EC24F0780EA3A7200E8BEC23F0000E35
:1032C000F86E520EF76EAC0EF66E46EC24F0000E61
:1032D000F86E530EF76E1A0EF66E43EC24F0780E6D
:1032E000A3A9200E8BEC23F0000EF86E520EF76EA1
:1032F000AC0EF66E46EC24F0000EF86E530EF76E30
:103300002A0EF66E43EC24F0780EA3AB200E8BEC65
:1033100023F0000EF86E520EF76EAC0EF66E46EC11
:1033200024F012003EEC23F0FFEC22F0000EF86EC9
:10333000540EF76E740EF66E43EC24F096EC22F009
:1033400062EC23F0FFEC22F0000EF86E540EF76EE4
:10335000740EF66E43EC24F096EC22F0F3EC18F0C9
:10336000000EF86E540EF76E740EF66E43EC24F0F9
:1033700096EC22F022EC19F0000EF86E540EF76E67
:10338000740EF66E43EC24F096EC22F050EC19F03B
:10339000000EF86E540EF76E740EF66E43EC24F0C9
:1033A00096EC22F029EC24F01200000EF86E520E7A
:1033B000F76EBA0EF66E43EC24F01EEC31F0ACC0A2
:1033C00018F0182A82EC3BF0020E376E386A7DEC5A
:1033D0003AF0000EF86E520EF76EAC0EF66E46EC3A
:1033E00024F0120029EC24F0C0EC21F0D4EC21F000
:1033F000E8EC21F006EC22F00B0E9E6155EC24F077
:103400000B0EA06167EC24F012008D6B8E6B9AC0DE
:1034100045F09BC046F09CC047F09DC048F09EC060
:1034200049F09FC04AF0A0C04BF0A1C04CF0A2C030
:103430004DF0A3C04EF0ACC04FF029EC24F0DEEC10
:1034400023F0000EF86E5E0EF76E460EF66E43EC3D
:1034500024F0000EF86E5E0EF76E5C0EF66E43EC16
:1034600024F0000EF86E5E0EF76E720EF66E43ECF0
:1034700024F001EC23F029EC24F0F2EC19F0000E1A
:10348000F86E520EF76EAE0EF66E43EC24F01EECA4
:1034900031F0ACC018F0182A82EC3BF0020E376E07
:1034A000386A7DEC3AF0000EF86E520EF76EAC0EF4
:1034B000F66E46EC24F028EC09F012E006E2AC2BA4
:1034C000140EAC6301D0AC6B05D0AC07ACAF02D02E
:1034D000130EAC6F5B6A29EC24F03BEC04F0CDD703
:1034E000F4EC22F0E8E3DEEC23F096EC22F0010E9F
:1034F000446201D053D0020E446201D04FD00B0E73
:10350000446201D004D00C0E446201D000D045C00A
:103510009AF046C09BF047C09CF048C09DF049C05F
:103520009EF04AC09FF04BC0A0F04CC0A1F04DC02F
:10353000A2F04EC0A3F04FC0ACF03BEC04F0446AE4
:103540003AEC1FF01200A76702D0000E22D0010E45
:10355000A76302D00B0E1DD0020EA76302D0400E4F
:1035600018D0030EA76302D04B0E13D0040EA7632E
:1035700002D0140E0ED0050EA76302D01F0E09D084
:10358000060EA76302D0540E04D0070EA76301D025
:103590005F0E31EC24F0DBEC23F0120029EC24F078
:1035A000A76BF2EC19F0A3EC1AF028EC09F009E093
:1035B00004E26DEC1BF05B6AF4D7ADEC1BF05B6AC8
:1035C000F0D7F4EC22F0F1E396EC22F0020E446224
:1035D00015D0A72B050EA76304D00A0E9E6501D057
:1035E000A72B070EA76304D00A0EA06501D0A72B56
:1035F000070EA76501D0A76B446AD3D7010E4462BA
:1036000001D00DD0020E446201D009D00B0E4462ED
:1036100001D07DD70C0E446201D079D712000F0E75
:103620009E6301D003D00F0EA06303D129EC24F0D8
:10363000000EF86E5E0EF76E460EF66E43EC24F04A
:10364000000EF86E610EF76E280EF66E43EC24F055
:10365000000EF86E540EF76E480EF66E43EC24F032
:10366000A2C018F0D6EC16F043EC16F028EC09F0E6
:1036700022E0A2C018F003E20A0E182602D00A0EB9
:10368000185E0F0E186003D00F0E186E10D0190EB2
:10369000186202D0140E186E550E186202D0500E29
:1036A000186E5F0E186403D05F0E186E00D018C03D
:1036B000A2F05B6AD5D7F4EC22F0D8E3DEEC23F07D
:1036C00096EC22F0010E446201D0B3D0020E4462A7
:1036D00001D0AFD087EF1AF01200A76705D09A2B60
:1036E0000A0E9A6501D09A6B010EA76305D09B2B39
:1036F0000A0E9B6501D09B6B020EA76305D09C2B25
:103700000A0E9C6501D09C6B030EA76305D09D2B10
:103710000A0E9D6501D09D6B040EA76305D09E2BFC
:10372000120E9E6501D09E6B050EA76305D09F2BE0
:103730000A0E9F6501D09F6B060EA76305D0A02BD4
:10374000120EA06501D0A06B070EA76305D0A12BB8
:103750000A0EA16501D0A16B1200A76705D09A07D8
:103760009AAF02D00A0E9A6F010EA76305D09B078D
:103770009BAF02D00A0E9B6F020EA76305D09C0779
:103780009CAF02D00A0E9C6F030EA76305D09D0765
:103790009DAF02D00A0E9D6F040EA76305D09E0751
:1037A0009EAF02D0120E9E6F050EA76305D09F0735
:1037B0009FAF02D00A0E9F6F060EA76305D0A00729
:1037C000A0AF02D0120EA06F070EA76305D0A1070D
:1037D000A1AF02D00A0EA16F1200A76702D0480E57
:1037E00023D0010EA76302D0470E1ED0020EA7639E
:1037F00002D0460E19D0030EA76302D0450E14D096
:10380000040EA76302D0440E0FD0050EA76302D0AA
:10381000430E0AD0060EA76302D0420E05D0070E53
:10382000A76302D0410E00D031EC24F0DBEC23F092
:103830001200A76B29EC24F0000EF86E5E0EF76EF6
:10384000880EF66E43EC24F0000EF86E540EF76E00
:10385000480EF66E43EC24F0000EF86E520EF76E32
:10386000B60EF66E43EC24F0300EA3BF310E8BEC97
:1038700023F0300EA3BD310E8BEC23F0300EA3BB32
:10388000310E8BEC23F0300EA3B9310E8BEC23F00C
:10389000300EA3B7310E8BEC23F0300EA3B5310EF2
:1038A0008BEC23F0300EA3B3310E8BEC23F0300EF3
:1038B000A3B1310E8BEC23F0000EF86E520EF76EB2
:1038C000AC0EF66E46EC24F0B7EC1CF0EDEC1BF001
:1038D00028EC09F004E097EC1CF05B6ABDD7F4EC2F
:1038E00022F0F6E3DEEC23F096EC22F0010E4462C7
:1038F0000AD031EC26F0D7EC03F03BEC04F029ECD5
:1039000024F0446A13D0020E446206D0A72B080E9E
:10391000A76301D0A76BA0D70B0E446202D087EF3C
:103920001AF00C0E446202D087EF1AF01200A7675B
:1039300001D0A371010EA76301D0A373020EA76388
:1039400001D0A375030EA76301D0A377040EA7636C
:1039500001D0A379050EA76301D0A37B060EA76350
:1039600001D0A37D070EA76301D0A37F1200A76734
:1039700013D0A3B109D0000EF86E5E0EF76E9E0E46
:10398000F66E43EC24F008D0000EF86E5E0EF76E73
:10399000B40EF66E43EC24F0010EA76313D0A3B36C
:1039A00009D0000EF86E5E0EF76ECA0EF66E43EC8E
:1039B00024F008D0000EF86E5E0EF76EE00EF66E84
:1039C00043EC24F0020EA76313D0A3B509D0000E78
:1039D000F86E5E0EF76EF60EF66E43EC24F008D02D
:1039E000000EF86E5F0EF76E0C0EF66E43EC24F0D0
:1039F000030EA76313D0A3B709D0000EF86E5F0EB5
:103A0000F76E220EF66E43EC24F008D0000EF86E2E
:103A10005F0EF76E380EF66E43EC24F0040EA763CB
:103A200013D0A3B909D0000EF86E5F0EF76E4E0EDC
:103A3000F66E43EC24F008D0000EF86E5F0EF76EC1
:103A4000640EF66E43EC24F0050EA76313D0A3BBFF
:103A500009D0000EF86E5F0EF76E7A0EF66E43EC2C
:103A600024F008D0000EF86E5F0EF76E900EF66E22
:103A700043EC24F0060EA76302D0B7EC28F0070E43
:103A8000A76302D0B7EC28F0120029EC24F0DEEC9A
:103A900023F0000EF86E5F0EF76EE80EF66E43EC44
:103AA00024F0000EF86E5F0EF76EFE0EF66E43EC1D
:103AB00024F0000EF86E600EF76E140EF66E43ECF6
:103AC00024F0000EF86E540EF76E480EF66E43ECBE
:103AD00024F001EC23F096EC22F0010E446220D099
:103AE000B7EC28F0FF0E546E000EF86E820EF76EE3
:103AF0005C0EF66E04EE00F004000900F550EE6E68
:103B0000542EFAD7000E066EFF0E546E04EE00F02F
:103B1000E7EC26F029EC24F009EC23F0FF0000D0BC
:103B200029EC24F03D82120029EC24F0000EF86EFE
:103B3000600EF76E2A0EF66E43EC24F0000EF86E5F
:103B4000600EF76E400EF66E43EC24F0000EF86E39
:103B5000600EF76E560EF66E43EC24F009EC23F07F
:103B600029EC24F03D821200DEEC23F029EC24F055
:103B7000000EF86E540EF76EF80EF66E43EC24F05D
:103B8000000EF86E550EF76E0E0EF66E43EC24F036
:103B900005EC23F029EC24F0DEEC23F07BC26EF080
:103BA0007CC26FF07DC26BF07EC26CF07FC270F0A1
:103BB00080C271F07BC261F07CC262F07BC263F0B4
:103BC0007CC264F0656B7DC266F07EC267F07DC228
:103BD00068F07EC269F06A6B7FC25CF080C25DF003
:103BE0007FC25EF080C25FF0606B7BC274F07CC20B
:103BF00075F07DC272F07EC273F07FC276F080C233
:103C000077F03BEC01F00BEC01F095EC01F01BECD4
:103C100001F0EBEC00F075EC01F02BEC01F0FBECAB
:103C200000F085EC01F0186A196A1A6A1B6A1C6AAE
:103C300018C03FF219C040F21AC041F21BC042F254
:103C40001CC043F2A6EC37F032C03AF233C03BF26C
:103C500034C03CF235C03DF236C03EF23AC253F2B7
:103C60003BC254F23CC255F23DC256F23EC257F23C
:103C70003FC258F240C259F241C25AF242C25BF20C
:103C800043C25CF23E8A8CEC22F00A0E576EDEECE8
:103C900023F00A0E566E0A0E31EC24F02A0E3DB4C3
:103CA000200E8BEC23F04A0E31EC24F02A0E3DA4BA
:103CB000200E8BEC23F03D74F4EC22F045E20A0E6A
:103CC0009E6504D0E2EC07F055EC24F00A0EA065E6
:103CD00004D025EC08F067EC24F0B16703D01EECAB
:103CE00003F005D0010EB16302D00EEC03F02DEC11
:103CF00025F0B06703D0A4EC02F01DD0010EB06334
:103D000003D094EC02F017D0020EB06303D0B4ECF1
:103D100002F011D0030EB06303D0D4EC02F00BD04C
:103D2000040EB06303D0F0EC02F005D0050EB063D2
:103D300002D0FFEC02F040EC25F00BEC23F0562E05
:103D4000BBD7572EA4D702D093EC22F0ADA502D05A
:103D5000896B8A6BA5EC01F079EC24F03E9A120095
:103D6000140E31EC24F0DBEF23F08D6B8E6BACC0C6
:103D700045F029EC24F0C0EC21F0D4EC21F0E8EC83
:103D800021F006EC22F00B0E9E6155EC24F00B0E98
:103D9000A06167EC24F0000EF86E520EF76EAE0EC6
:103DA000F66E43EC24F01EEC31F0ACC018F0182A8B
:103DB00082EC3BF0020E376E386A7DEC3AF0000E72
:103DC000F86E520EF76EAC0EF66E46EC24F0000E56
:103DD000F86E520EF76EB20EF66E43EC24F0A3515D
:103DE0003AEC24F0000EF86E520EF76EAC0EF66E42
:103DF00046EC24F028EC09F012E006E2AC2B140E9D
:103E0000AC6301D0AC6B05D0AC07ACAF02D0130EE5
:103E1000AC6F5B6A29EC24F03BEC04F0ACD7F4EC1B
:103E200022F0E8E3DEEC23F096EC22F0010E44628F
:103E300001D00CD0020E446201D008D00B0E4462B7
:103E400001D013D00C0E446210D00FD0F3EC18F058
:103E500001EC23F022EC19F001EC23F050EC19F006
:103E600001EC23F031EC26F004D045C0ACF03AEC84
:103E70001FF01200000EF86E530EF76E500EF66E25
:103E800043EC24F0000EF86E530EF76E660EF66EDD
:103E900043EC24F0000EF86E530EF76E7C0EF66EB7
:103EA00043EC24F0FFEC22F029EF24F0B1C045F000
:103EB00029EC24F0000EF86E550EF76EA80EF66E83
:103EC00043EC24F0000EF86E530EF76E3A0EF66EC9
:103ED00043EC24F0DEEC23F0B16710D0000EF86E56
:103EE000560EF76E160EF66E43EC24F0000EF86ECA
:103EF000560EF76E2C0EF66E43EC24F0010EB163F5
:103F000010D0000EF86E560EF76E420EF66E43ECB1
:103F100024F0000EF86E560EF76E580EF66E43EC57
:103F200024F0B0EC1EF028EC09F00DE006E2B12B15
:103F3000010EB16501D0B16B05D0B107B1AF02D0B0
:103F4000010EB16FC7D7F4EC22F0EBE3DEEC23F007
:103F500096EC22F0030E446006D0010E446203D0BA
:103F6000EBEC25F004D045C0B1F03AEC1FF01200A4
:103F7000B0C045F029EC24F0000EF86E560EF76E36
:103F8000000EF66E43EC24F0000EF86E530EF76E42
:103F90003A0EF66E43EC24F0DEEC23F0B06710D05E
:103FA000000EF86E560EF76E6E0EF66E43EC24F0B1
:103FB000000EF86E560EF76E840EF66E43EC24F08B
:103FC000010EB06310D0000EF86E560EF76E9A0E0A
:103FD000F66E43EC24F0000EF86E560EF76EB00E3F
:103FE000F66E43EC24F0020EB06310D0000EF86EB3
:103FF000560EF76EC60EF66E43EC24F0000EF86E09
:10400000560EF76EDC0EF66E43EC24F0030EB06332
:1040100010D0000EF86E560EF76EF20EF66E43ECF0
:1040200024F0000EF86E560EF76E580EF66E43EC46
:1040300024F0040EB06310D0000EF86E570EF76E29
:10404000080EF66E43EC24F0000EF86E560EF76E76
:10405000580EF66E43EC24F0050EB06310D0000E3F
:10406000F86E570EF76E1E0EF66E43EC24F0000E3F
:10407000F86E560EF76E580EF66E43EC24F0B0EC68
:104080001EF028EC09F00DE006E2B02B050EB0653D
:1040900001D0B06B05D0B007B0AF02D0050EB06F45
:1040A0007BD7F4EC22F0EDE3DEEC23F096EC22F08B
:1040B000030E44600AD0010E446207D0FDEC25F0E7
:1040C000020EB06306D0FBEF17F045C0B0F03AEC3B
:1040D0001FF01200000EF86E520EF76E040EF66E10
:1040E00046EC24F063C018F064C019F01AD0000E3A
:1040F000F86E520EF76E0A0EF66E46EC24F068C0AB
:1041000018F069C019F00DD0000EF86E520EF76E5F
:10411000100EF66E46EC24F05EC018F05FC019F089
:1041200000D01A6A1B6A1C6A82EC3BF0040E376EE0
:10413000386A51EF3AF0000EF86E510EF76EC20E6B
:10414000F66E46EC24F049C24BF14AC24CF14BC228
:104150004DF14CC24EF14DC24FF126D0000EF86E1B
:10416000510EF76EC40EF66E46EC24F044C24BF1CD
:1041700045C24CF146C24DF147C24EF148C24FF123
:1041800013D0000EF86E510EF76EC60EF66E46ECAA
:1041900024F04EC24BF14FC24CF150C24DF151C20E
:1041A0004EF152C24FF100D03D0E8BEC23F0F7ECF4
:1041B0003CF06CEC3DF0A3B116D066EC00F013E3DC
:1041C000186A196A1A6A1B6A1C6A18C050F119C069
:1041D00051F11AC052F11BC053F11CC054F1030E2F
:1041E000186E18C05AF13CEF3FF03EAA09D0000EFD
:1041F000F86E510EF76EAA0EF66E46EC24F01CD047
:10420000000EF86E510EF76EA40EF66E46EC24F01A
:1042100058C22DF059C22EF05AC22FF05BC230F0B6
:104220005CC231F09BEC3BF0040E376E020E386E30
:104230003CEC3BF07DEC3AF012003EAA09D0000EB7
:10424000F86E510EF76EB80EF66E46EC24F024D0E0
:10425000000EF86E510EF76EB40EF66E46EC24F0BA
:1042600053C22DF054C22EF055C22FF056C230F07A
:1042700057C231F09BEC3BF0030E376E010E386EE7
:104280003CEC3BF07DEC3AF0000EF86E620EF76EFF
:10429000180EF66E46EC24F01200000EF86E510E69
:1042A000F76EC20EF66E46EC24F049C24BF14AC2DC
:1042B0004CF14BC24DF14CC24EF14DC24FF10CEFDF
:1042C0003FF0000EF86E510EF76EC40EF66E46EC1F
:1042D00024F044C24BF145C24CF146C24DF147C2F5
:1042E0004EF148C24FF10CEF3FF0000EF86E510E48
:1042F000F76EC60EF66E46EC24F04EC24BF14FC27E
:104300004CF150C24DF151C24EF152C24FF10CEF7F
:104310003FF0AB6702D0DEDE32D0010EAB6302D0DD
:10432000E6DE2DD0020EAB6302D0EEDE28D0030E07
:10433000AB6302D0B2DF23D0040EAB6302D0C1DF87
:104340001ED0050EAB6302D0D0DF19D0060EAB63D2
:1043500002D0F1DE14D0070EAB6302D0FFDE0FD027
:10436000080EAB6302D00DDF0AD0090EAB6302D09A
:104370003CDF05D00A0EAB6302D05FDF00D0120035
:10438000DEEC23F0000E31EC24F09AC0ABF089ECA7
:1043900021F00B0E31EC24F09BC0ABF089EC21F046
:1043A0003EBC65EC05F01200DEEC23F0400E31EC73
:1043B00024F09CC0ABF089EC21F04B0E31EC24F0E2
:1043C0009DC0ABF089EC21F03EBC65EC05F012001D
:1043D000DEEC23F00B0E9E6112D0140E31EC24F0B3
:1043E0009EC0ABF089EC21F01F0E31EC24F09FC091
:1043F000ABF089EC21F03EBC65EC05F01200140E28
:1044000031EC24F09EC0ABF024EF22F0DEEC23F080
:104410000B0EA06112D0540E31EC24F0A0C0ABF012
:1044200089EC21F05F0E31EC24F0A1C0ABF089ECF7
:1044300021F03EBC65EC05F01200540E31EC24F086
:10444000A0C0ABF024EF22F00B0EAB6308D0000E3F
:10445000F86E520EF76E160EF66E46EC24F00C0E49
:10446000AB6308D0000EF86E520EF76E1A0EF66EA1
:1044700046EC24F00D0EAB6308D0000EF86E520E21
:10448000F76E220EF66E46EC24F00E0EAB6308D0EB
:10449000000EF86E520EF76E1E0EF66E46EC24F00D
:1044A0000F0EAB6317D0000EF86E520EF76E260E8D
:1044B000F66E46EC24F0A2C018F08BEC33F00AEC58
:1044C00035F0EFEC37F09BEC3BF0010E376E386ABD
:1044D0007DEC3AF0100EAB6308D0000EF86E520E71
:1044E000F76E2A0EF66E46EC24F0110EAB6308D080
:1044F000000EF86E520EF76E2E0EF66E46EC24F09D
:10450000120EAB6308D0000EF86E520EF76E320E2C
:10451000F66E46EC24F0120033DF46DF59DF76D723
:1045200063D8FEE3120060D8FEE21200F9DF446AAD
:104530000FEC23F081B603D0010E446E05D081B498
:1045400003D0020E446E00D00A0E546E0BEC23F022
:10455000F4EC22F048E3542EF9D70A0E442629EC55
:1045600024F00B0E44622CD0B26709D0000EF86E16
:10457000530EF76E9E0EF66E43EC24F02FD0010E14
:10458000B26309D0000EF86E530EF76EA80EF66EE9
:1045900043EC24F023D0020EB26309D0000EF86E73
:1045A000530EF76EB40EF66E43EC24F017D0000EE7
:1045B000F86E530EF76E920EF66E43EC24F00ED0AA
:1045C0003EB804D00C0E446200D008D0000EF86E45
:1045D000530EF76EA80EF66E43EC24F093EC22F027
:1045E00029EC24F03D821200040081B601D005D0F0
:1045F00081B401D002D0D8901200D880120001EC12
:1046000023F007EC23F007EC23F007EC23F0FA0E7D
:1046100009D0C80E07D0640E05D0320E03D00A0EA2
:1046200001D0010E0400426EC80E406E150E416EA0
:10463000402EFED7412EFCD7422EF6D712008B9A81
:104640008B968B98EADF300ECAD8EBDF300EC7D8D6
:10465000E8DF300EC4D8E5DF200EC1D8E0DF290E38
:10466000AED8080EACD8060EAAD8010EA8D8020EF5
:10467000A6D80C0EA4D870D8A1D81200DEEC23F076
:10468000E8D8000EF86E610EF76E580EF66E43EC29
:1046900024F0000EF86E610EF76E6E0EF66E43ECAF
:1046A00024F0000EF86E610EF76E840EF66E43EC89
:1046B00024F0000EF86E610EF76E9A0EF66E43EC63
:1046C00024F01200DEEC23F0C4D8000EF86E610E68
:1046D000F76E580EF66E43EC24F0000EF86E610E85
:1046E000F76E6E0EF66E43EC24F0000EF86E610E5F
:1046F000F76EB00EF66E43EC24F0000EF86E610E0D
:10470000F76EC60EF66E43EC24F0120000000000B7
:10471000000000001200086E74D808508B8686ECEA
:1047200023F08B9886EC23F08B9A86EC23F0F00B29
:1047300056D80838F00B53D0086E0846084608468D
:1047400060D8085040093BD8080E546E0900F55057
:10475000E2DF542EFBD71200000EF86E470EF76E04
:10476000760EF66E080E556E566A5650E5DF562ADE
:10477000552EFBD7120000001818181B000000006F
:104780001B1B1B1B000000000303031B00000E117A
:104790000E00001F00000E110E000D1513000E116B
:1047A0000E000A15150000000000101B100000008C
:1047B0000000001B0000C0C0E8FF01D00C0E086E16
:1047C00020D80850F00B8B9686EC23F08B9886EC63
:1047D00023F08B9A86EC23F002D80838F00B040003
:1047E00081B0010981B2020981B4040981B60809C6
:1047F000816E86EC23F08B8A86EC23F08B9A86EF11
:1048000023F00400818E86EC23F0938E86EC23F057
:104810008B9686EC23F08B885868584E15D086EC22
:1048200023F03A9686EC23F08B8A86EC23F081AE57
:104830003A8686EC23F08B9A86EC23F08B8A86EC02
:1048400023F08B9A3AA6E9D7939E8B9886EC23F0B7
:104850001200010EB4DF020EB2D7800EB0D7C00E28
:10486000AED78009ACD7200E56D7546EFCDF542E3D
:10487000FDD71200096E093812EC00F04CDF095028
:1048800012EC00F048D70900F550EBDF0900F550B5
:1048900002E041DFFBD712000900F55002E002D828
:1048A000FBD71200E8CFDEFF12003F923EBE3F82F0
:1048B00079C0A4F07BC0A5F0ADA7A56B170EA66FBD
:1048C0003DB81DEC27F03DA89AEC27F012003F926E
:1048D0003FB03F827CC0A4F07EC0A5F0ADA9A56B1F
:1048E000570EA66F3DBA1DEC27F03DAA9AEC27F0B3
:1048F0001200DBDFECD7F00ED36E400E9B6E0F0183
:10490000806A896A070E386F0F0E926E816A8A6A12
:10491000000E396F0F0E936E826A8B6A800E946E52
:10492000000E3A6F040EC16EB60EC06E000ED06E51
:10493000F00EF26E000EF16E000EF06E010E9D6E26
:10494000000EA06E000EA36E310ECD6E000EBA6E7C
:10495000000EB16EB10ECF6EE00ECE6E310ECD6E8A
:10496000010E9D6E000EA06E4D0ED66E070ED56E1A
:10497000F60ED76E3C0ED66E00011200546A00EEA1
:1049800000F0EE6A542EFDD7040E556E01EE00F0D5
:10499000EE6A542EFDD7552EFBD712001200C5D952
:1049A000B2D9D5D968D93BEC04F053D9E2D90BD9A7
:1049B0001CD92DD972D983D994D9CEEC04F039D928
:1049C000EAD929EC00F037EC00F01200FF0EBB6EC4
:1049D0000C0EBD6E926B936B40D80C0E666E986B8E
:1049E000996B4ED8000EBA6E030EBC6EBA841200DC
:1049F000ADB305D094C092F095C093F02CD09751F0
:104A0000955D02E19651945DD8A401D007D09551EF
:104A1000975D02E19451965DD8B007D0640E8B6F1C
:104A200094C096F095C097F012D08B6715D08C6724
:104A300013D0140E186E000E196E1850965F195090
:104A4000975B0A0E8C6F97AF02D0966B976B96C0F0
:104A500092F097C093F001D8120092C054F093C026
:104A600055F0D89055325432D8905532543254C003
:104A7000BEFFBD98BD9A92B1BD8892B3BD8A1200A7
:104A800098C054F099C055F0D89055325432D8900F
:104A90005532543254C067FF6698669A98B166885A
:104AA00098B3668A12002A0E066E39D0340E066E4E
:104AB00036D03E0E066E33D0480E066E30D0520E03
:104AC000066E2DD05C0E066E2AD0660E066E27D0BE
:104AD000700E066E24D07A0E066E21D0840E066EFD
:104AE0001ED08E0E066E1BD0980E066E18D0A20E2B
:104AF000066E15D0AC0E066E12D0B60E066E0FD036
:104B0000C00E066E0CD0CA0E066E09D0D40E066E0C
:104B100006D0DE0E066E03D0E80E066E00D00A0E3A
:104B2000546E00EE9AF0E7EC26F009EF23F02A0E1F
:104B3000066E39D0340E066E36D03E0E066E33D079
:104B4000480E066E30D0520E066E2DD05C0E066EEC
:104B50002AD0660E066E27D0700E066E24D07A0E0E
:104B6000066E21D0840E066E1ED08E0E066E1BD0F1
:104B7000980E066E18D0A20E066E15D0AC0E066EFC
:104B800012D0B60E066E0FD0C00E066E0CD0CA0E36
:104B9000066E09D0D40E066E06D0DE0E066E03D069
:104BA000E80E066E00D00A0E546E00EE9AF0FCEF8E
:104BB00026F0260E066E020E546E00EEAEF0E7EC06
:104BC00026F009EF23F0260E066E020E546E00EE5C
:104BD000AEF0FCEF26F01A0E066E010E546E00EEDB
:104BE000B1F0E7EC26F009EF23F01A0E066E010E85
:104BF000546E00EEB1F0FCEF26F01B0E066E010EB7
:104C0000546E00EEB0F0E7EC26F009EF23F01B0E37
:104C1000066E010E546E00EEB0F0FCEF26F0210E91
:104C2000066E010E546E00EEC0F0E7EC26F009EFC0
:104C300023F0210E066E010E546E00EEC0F0FCEF64
:104C400026F01C0E066E050E546E02EE71F0E7EFB4
:104C500026F01C0E066E050E546E02EE71F0FCEF8F
:104C600026F0190E066E010E546E00EEACF0E7EC65
:104C700026F009EF23F0190E066E010E546E00EEB9
:104C8000ACF0FCEF26F0000E066E0A0E546E02EE3B
:104C900017F0E7EC26F009EF23F0000E066E0A0E7F
:104CA000546E02EE17F0FCEF26F00A0E066E0A0EA6
:104CB000546E02EE21F0E7EC26F009EF23F00A0E25
:104CC000066E0A0E546E02EE21F0FCEF26F0140E72
:104CD000066E050E546E02EE6CF0E7EC26F009EF5E
:104CE00023F0140E066E050E546E02EE6CF0FCEF0F
:104CF00026F0290E066E010E546E02EE02F0E7EC6D
:104D000026F009EF23F0290E066E010E546E02EE16
:104D100002F0FCEF26F0220E066E020E546E02EE3A
:104D200000F0E7EC26F009EF23F0220E066E020EEB
:104D3000546E02EE00F0FCEF26F0240E066E020E1A
:104D4000546E02EE03F0E7EC26F009EF23F0240E98
:104D5000066E020E546E02EE03F0FCEF26F0250EF6
:104D6000066E010E546E00EEADF0E7EC26F009EF92
:104D700023F0250E066E010E546E00EEADF0FCEF32
:104D800026F0280E066E010E546E02EE95F0E7EC4A
:104D900026F009EF23F0280E066E010E546E02EE87
:104DA00095F0FCEF26F0A6B2FED706C0A9FF07C01B
:104DB000A8FFA69EA69CA684F29EF2BEFED7550E24
:104DC000A76EAA0EA76EA682F28EA6941200040009
:104DD000EECF07F0D3EC26F0062A542EF8D794EF46
:104DE0001DF01200A6B2FED706C0A9FFA69EA69C83
:104DF000A680A850076E12000400F2EC26F007C04F
:104E0000EEFF062A542EF8D712001D0E0DD0190EF3
:104E10000BD0150E09D0110E07D00D0E05D0090EBE
:104E200003D0050E01D0010EC26EC282C2B2FED7FF
:104E3000C4CF5AF0C3CF59F01200DEEC23F007D8EC
:104E4000A4C045F04FD8A5C045F04CD80ED0110EE7
:104E5000546E03EE20F0070EE8CFEEFF542EFBD782
:104E6000060E186E18C02FF312003FA22ED08E67C8
:104E70002CD08D532AE123EE29F05B0E52EC24F066
:104E800071C22DF072C22EF073C22FF074C230F0D6
:104E900075C231F008EC05F0E3EC35F02DC04BF1B4
:104EA0002EC04CF12FC04DF130C04EF131C04FF14A
:104EB000F7EC3CF06CEC3DF09AEC40F023EE2EF079
:104EC000CBEC40F05D0E52EC24F0A65131EC24F016
:104ED000110E546E03EE20F0EE508BEC23F0542EA6
:104EE000FBD7120003EE20F045C01DF0220E1D641A
:104EF00003D0220E1D6E05D01D2AD8901D321DC074
:104F000054F0EE50542EFDD71E6EED50070E1E626B
:104F100001D003D0060E1E6205D0020E45B0000E71
:104F2000EF6E07D0000E1E6204D0010E45B0000ED9
:104F3000EF6E1200DEEC23F08ADFA4C01DF0220E1B
:104F40001D6402D0220E1D6ED8901D321DC054F07B
:104F500003EE20F0545204E0010EEE6E542EFCD706
:104F6000A4A102D0000EEE6EA5C045F0BBDF7DD738
:104F7000140E546E03EE00F081CFE8FF120BE8CF61
:104F8000EEFF86EC23F0542EF7D70DD0140E546E9E
:104F900003EE00F081CFE8FF030BE8CFEEFF86ECD5
:104FA00023F0542EF7D7B56BB66BB76BB86BB96BF4
:104FB000BA6BBB6BBC6BBD6BBE6B130E546E03EE5A
:104FC00000F0EECFB5F0EECFBEF0BD670AD0BEC0A8
:104FD000E8FFB55D02E1B62B27D0BD2BBEC0B7F010
:104FE00023D0010EBD630AD0BEC0E8FFB75D02E169
:104FF000B82B1AD0BD2BBEC0B9F016D0020EBD63BF
:105000000AD0BEC0E8FFB95D02E1BA2B0DD0BD2BBE
:10501000BEC0BBF009D0030EBD6306D0BEC0E8FF22
:10502000BB5D02E1BC2B00D0542ECDD7B6C0BDF085
:10503000B5C0B4F0B851BD5DD8B004D0B8C0BDF0B3
:10504000B7C0B4F0BA51BD5DD8B004D0BAC0BDF09D
:10505000B9C0B4F0BC51BD5DD8B004D0BCC0BDF087
:10506000BBC0B4F01200006ED8CF01F0E0CF02F068
:105070009EA048D09E907F677F07806780078167EA
:105080008107826782078B678B078C678C07836732
:1050900002D0845306E083078329D8B48407D8B4A8
:1050A00083538867880787678707856702D0865399
:1050B00006E085078529D8B48607D8B485538D675F
:1050C00002D08E5306E08D078D29D8B48E07D8B450
:1050D0008D53896702D08A5306E089078929D8B49D
:1050E0008A07D8B489538F6702D0905306E08F07A0
:1050F0008F29D8B49007D8B48F53B10ECF6EE00E7D
:10510000CE6E22D0F2A216D0F292F298D58EC6ECD4
:1051100027F0ADA103D0F17CF1AC06D0B4A302D04E
:105120005B2A07D05B0605D0B4B302D05B2A01D05E
:105130005B060AD0F2A408D0F294F288D59EF60E4F
:10514000D76E3C0ED66E00D002C0E0FF005001C00A
:10515000D8FF1000036ED8CF04F0E0CF05F005C0F3
:10516000E0FF035004C0D8FF1000540E05D0140E09
:1051700003D0400E01D0000E31EC24F0000EF86E8A
:10518000510EF76E8E0EF66E46EC24F012002020C3
:10519000202020202020202020202020202020200F
:1051A000202000005357523D00005357523D202D00
:1051B0002C2D2D00524C3D00524C3D202D2C2D64A9
:1051C0004200500046005200002D2D2D20426172F9
:1051D00067726170682F50574D202D2D2D00402D86
:1051E0002D2064426D204C6576656C206C696D697C
:1051F00074202D00145B000064426D5D203D205B37
:1052000000005D00414443703D00414443663D0061
:10521000414443723D005045500020204600524C0E
:105220003100524C320053570000202052005231BE
:1052300030005232300014424731000054424732AD
:1052400000004D5B7365635D0000002D2D2D2D2D3D
:1052500020414443203064426D202D2D2D2D2D0002
:10526000002D2D2D2D20414443202D333064426DDF
:10527000202D2D2D2D004041444320203064426DCF
:105280003A00144144432D333064426D3A00405695
:10529000616C75653A0014526F74617279206B65A8
:1052A000793D537465702020202020005D005B5BF9
:1052B00000001B5B0000405B000000446973706CE1
:1052C0006179205661723A205B0040506F776572B9
:1052D000206D696E2E203A205B00145357522F52D6
:1052E0004C6D696E2E203A205B0000636F75706C08
:1052F0002E206C6F73733A205B004042472D53574A
:10530000526D617820203A205B00004156472050C2
:105310004550202020203A205B0040415647205035
:10532000666F72772E203A205B001441564720505A
:1053300072657475726E3A205B00403D3D3D3D3DA7
:105340003D3D3D3D3D3D3D3D3D3D3D3D3D3D3D00CA
:10535000003D3D3D3D3D2046756E6374696F6E2096
:105360003D3D3D3D3D00402D2D2D2D2061626F7254
:10537000746564202121202D2D2D2D00143D3D3DEF
:105380003D3D3D3D3D3D3D3D3D3D3D3D3D3D3D3D4D
:105390003D00004B6579206C6F6E67202000005344
:1053A000455455502D3E00000041424F525420209C
:1053B0002D3E0000004368616E6765202D3E0000B1
:1053C0000041444355666F72772E3A004041444392
:1053D0005566504550203A0000414443557265746B
:1053E0002E203A00144C6576656C313A20306442C8
:1053F0006D202020202020202000144C6576656C34
:10540000323A202D333064426D20202020202000AD
:10541000003D3D2041443833303720466F7277617C
:105420007264203D3D00003D3D204144383330371B
:105430002052657475726E203D3D3D00406D6B7865
:105440003A00146D6B793A005473686F72743D4F73
:105450004B206C6F6E673D427265616B2000547328
:10546000686F72743D4F4B206C6F6E673D4368618F
:105470006E676500544B6579202D3E206E6578740B
:1054800020202020202020202000544B6579202D32
:105490003E2061626F727420202020202020200096
:1054A000003D3D3D3D3D3D204D656E7565203D3DDA
:1054B0003D3D3D3D3D00405B315D52657472696527
:1054C0007665204D61782076616C2E001420206F67
:1054D0006620746865206C6173742078206D696E35
:1054E0002E0054202041626F7274204B65792D6C20
:1054F0006F6E672020202000003D20526574726985
:10550000657665204D61782076616C2E3D001445EE
:105510007869742077697468204B65792120202090
:1055200020202000405B325D20446973706C6179FB
:105530002056617269616E7473001420202020442B
:105540006973706C61792076617269616E74730041
:105550005420202020312E2E782020202020202092
:10556000202020202000405B335D2050574D312DFE
:105570004F75747075742020202020001420202086
:105580002050455020616E642050666F72772E2047
:1055900020005420202020202020202020202020F7
:1055A0002020202020202000003D3D3D2050574D50
:1055B00031204F7574707574203D3D3D3D00405B5A
:1055C000345D2050574D322D4F7574707574202006
:1055D000202020001420524C2D333064622F3630AE
:1055E000644220302E2E3556200054205357522C22
:1055F0002050722C2050722B31302F3230644200F8
:10560000003D3D3D2050574D32204F7574707574EC
:10561000203D3D3D3D00143020506F776572205095
:1056200045502020202020202020200054202045EC
:105630006E76656C6F7065207065616B2020202030
:105640002000143120506F77657220666F72776189
:10565000726420202020200054202061626F757425
:1056600020415647202020202020202020001430D8
:105670002052657475726E204C6F737320286462BB
:10568000292020005420302E2E36306442202D3E1A
:1056900020302E2E35566F6C7400143120526574F4
:1056A00075726E204C6F737320286462292020006D
:1056B0005420302E2E33306442202D3E20302E2EAA
:1056C00035566F6C740014322053575220312C30F1
:1056D00020746F2020782C78202020005420312C3A
:1056E000302E2E782C782D3E20302E2E35566F6C95
:1056F0007400143320506F77657220526574757290
:105700006E202020202020001434205072657475F3
:10571000726E202B3130644220202020200014356E
:10572000205072657475726E202B323064422020D6
:1057300020202000003D3D3D3D3D3D20534554553A
:1057400050203D3D3D3D3D3D3D00405B305D2041B5
:10575000626F727420202020202020202020200032
:10576000405B315D2055666F72772E2063616C69F6
:105770006272617465001420204D656173757269F1
:105780006E6720626F6172642058320054202020BE
:105790002041443833303720494332202020202014
:1057A0002000405B325D205572657475726E206317
:1057B000616C69622E2020001420204D6561737594
:1057C00072696E6720626F617264205831005420E4
:1057D00020202041443833303720494331202020D5
:1057E00020202000405B335D2064697265632E20B9
:1057F000436F75706C657220200014202020206398
:105800006F75706C696E67206C6F73732020200059
:10581000542020202077696E64696E672073746558
:10582000656C20202000002D2D2D20646972656399
:105830002E436F75706C6572202D2D004020436FD4
:1058400075706C696E67206C6F7373202020202048
:105850002000145764673A001E3D0000405B345D31
:10586000204C434420446973706C61792054696D05
:105870006500142020202056616C7565205045502D
:105880002020202020202000542020202050722C76
:105890002053575220616E6420524C202000002D6E
:1058A000204C434420446973706C61792054696DC5
:1058B00065202D00405B355D20426172677261702A
:1058C000682020202020202020001420202020508C
:1058D00065616B26486F6C642054696D65202000FB
:1058E0005420202020202020202020202020202084
:1058F000202020202000002D2D2D2D2D20426172F2
:105900006772617068202D2D2D2D2D00405B365D56
:105910002056696577204D2E686561642D66772E67
:1059200020001420202020414443312C3220616E7D
:1059300064206D6B782020005420202020616E644C
:10594000206D6B792076616C756520202000405BAE
:10595000375D2056696577204D2E686561642D722C
:1059600065742E00405B385D2042617247722F5093
:10597000574D2054657374202000142020202042AD
:105980006172677261706820312F32202020200000
:105990005420202020616E642050574D20312F323A
:1059A000202020202000002D2D2042617247722FE0
:1059B00050574D2054657374202D2D0040424731BF
:1059C0002F323A004A50574D3A00405B395D205221
:1059D0006F7461727920656E632E54797065200052
:1059E000142020646966666572656E74207479702F
:1059F0006573202020005420526173742F53746506
:105A00007020726174696F2020202000002D2052C8
:105A10006F7461727920656E632E54797065202DE4
:105A20002D00405261737420322C20537465703104
:105A3000205B0000405B31305D204D61782E63615A
:105A40002E2D6F66662076616C0014202073746FB3
:105A5000726167652074696D6520616E6420200045
:105A6000542020434C52206F6E2F6F6666202020FA
:105A70002020202020000020534554204D61782E06
:105A800063612E2D6F66662076616C0040686F6CD6
:105A9000642074696D653A001456696577207468EE
:105AA000656E20434C52205B0000405B31315D202D
:105AB0004D616E75656C6C204D682E666F72770057
:105AC00014202063616C6962726174652077697467
:105AD000686F7574200054202052462D47656E650E
:105AE0007261746F7220202020202000405B3132D0
:105AF0005D204D616E75656C6C204D682E7265740D
:105B00002E00405B31335D2050574D205365747437
:105B1000696E677320202000142020706F696E74F6
:105B2000657220696E6572746961202020005420BE
:105B300020504550205065616B26486F6C642020D2
:105B400020202000002D2D2D2050574D205365740E
:105B500074696E6773202D2D2D004054696D657238
:105B6000503A0000145045502C5065616B26486F28
:105B70002E6C6F6E67205B00405B31345D204657B2
:105B80002D55706461746520202020202000142D84
:105B9000206C6F616420696E746F2074686520509A
:105BA00049432000542D20776974682050432D53B9
:105BB000572D3E55534220202000002D2D2D2D2005
:105BC000465720557064617465202D2D2D2D2D00B4
:105BD000405553422D436162656C20706C7567209F
:105BE000696E2020210014506C656173652050435C
:105BF0002D5357207374617274202100002D2D2DB8
:105C0000204E6F20426F6F746C6F61646572202D3F
:105C10002D00402D2D2D2D2020696E206D656D6F7E
:105C20007279202D2D2D2D00142D2D2D2D2D2D2073
:105C3000666F756E64202D2D2D2D2D2D2D00542D6C
:105C40002D2D2D2D2041626F72742121202D2D2D9F
:105C50002D2D2D00402D2048572066726F6D20504D
:105C60004320666F756E64202D00142D2D20557015
:105C70006461746520737461727473202D2D2D001E
:105C8000542D2D20506C65617365207761697421F6
:105C90002121202D2D00405B31355D205357522DA1
:105CA000446973706C61792D50574D001420204465
:105CB0006973706C61792072616E676520202020A5
:105CC000200054202073657420757020202020202F
:105CD0002020202020202000002D2D205357522D41
:105CE000446973706C61792D50574D202D00405BD5
:105CF00031365D205049432D5761746368646F6786
:105D00002020200014202052657374617274732067
:105D1000496E666F20212020200054202020202062
:105D20002020202020202020202020202020200093
:105D3000002D2D2D205049432D5761746368646FE9
:105D400067202D2D2D004052657374617274733A73
:105D50000000405B31375D20437572736F722074B1
:105D6000797065202020200014202054797065204F
:105D70006F6620636F7572736520202020005420A9
:105D80002073657420757021212020202020202080
:105D900020202000002D20437572736F7220534520
:105DA00054202D2D2D2D2D2D200040437572736F05
:105DB000722D3E414243000040437572736F722D55
:105DC0003E00405B31385D20496E666F2046697247
:105DD0006D77617265202000142020446174652C69
:105DE0002048572C204657202020202020005420D7
:105DF00020496E666F732020202020202020202044
:105E000020202000405B31395D20446973706C6153
:105E100079205661722E20202000142020656469AC
:105E2000742C207365742020202020202020200046
:105E3000542020202020202020202020202020202E
:105E4000202020202000002D20446973706C61798F
:105E50002056617269616E7465202D004020456E88
:105E6000636F6465723A2053656C656374696F6E25
:105E70002000142057616974212020202020202038
:105E80002020202020202000002D204665617475F0
:105E90007265732020202020202020202000142D37
:105EA00020506F776572204D696E696D756D204F5A
:105EB0004E202000142D20506F776572204D696EA2
:105EC000696D756D204F46462000142D20535752A2
:105ED0002F524C204D696E696D756D204F4E20001C
:105EE000142D205357522F524C204D696E696D75F9
:105EF0006D204F464600142D20636F75706C696EDF
:105F000067206C6F7373204F4E202000142D206388
:105F10006F75706C696E67206C6F7373204F4646A7
:105F20002000142D204156472050706570202020FD
:105F300020204F4646202000142D20415647205057
:105F400070657020202020204F4E20202000142D2E
:105F5000204156472050666F7277617264204F4629
:105F600046202000142D204156472050666F72773E
:105F7000617264204F4E20202000142D204156478E
:105F8000205072657475726E20204F4646202000A6
:105F9000142D20415647205072657475726E202072
:105FA0004F4E20202000405B32305D20446566610A
:105FB000756C742053657474696E670014202061D9
:105FC0006C6C20506172616D657465727320202065
:105FD0002000542020466163746F727920736574C9
:105FE00074696E6720202000002D2D2044656661B5
:105FF000756C742053657474696E67202D004020A1
:1060000020616C6C204461746573205345542020DA
:106010002020200014202020206174206465666107
:10602000756C7420202020202000003D3D3D3D2047
:10603000536176652044617461203D3D3D3D3D00E6
:10604000403D3D3D3D3D3D3D20746F203D3D3D3D4E
:106050003D3D3D3D3D00143D3D3D3D2050494320EB
:10606000456570726F6D203D3D3D3D00003D3D3DFD
:106070003D3D3D204E6F74696365203D3D3D3D3D96
:106080003D00402020506C65617365206E6F746523
:1060900020616E642020200014206172636869769C
:1060A000652074686520666F6C6C6F772E005420D5
:1060B0002032204144432076616C75657321212094
:1060C0002020200040202028302C3520746F2020F4
:1060D00031302073656329202000144C43446861EB
:1060E0006E673A001450574D68616E673A0014535A
:1060F000575220312C3020746F202000402020285F
:106100003020746F2020322C3520736563292020C5
:10611000200040205357522D52616E676520202089
:10612000202020202020200040205357522D426163
:106130007267726170682D52616E67652000405011
:1061400065616B26486F6C643A006D73656300008F
:10615000736563006D696E00003D205152502D50F3
:106160006F7765722D4D65746572203D3D00403D31
:106170003D3D20316D5720746F2031353057203D23
:106180003D3D3D00143D3D3D3D2028632920444CCC
:10619000344A414C203D3D3D3D00543D3D3D3D2078
:1061A00032362E30322E32303231203D3D3D3D00F0
:1061B000143D2048573A2056657273696F6E20313E
:1061C0002E7878203D00543D2046573A205665727F
:1061D00073696F6E20312E3130203D002D2D2D0042
:1061E000494E46006D570000755700006E5700007D
:1061F00070570000665700006157000057200000EC
:106200006B570000205600006D56000075560000C8
:106210006E56000064426D0064420000737300001B
:1062200013D806D8136A146A156A166A176A120018
:106230000E6A0F6A106A116A126A1200186A196AE5
:106240001A6A1B6A1C6A1200F9DF1D6A1E6A1F6A3D
:10625000206A216A12002D6A2E6A2F6A306A316A1A
:1062600012000EC132F00FC133F010C134F011C171
:1062700035F012C136F012000EC12DF00FC12EF014
:1062800010C12FF011C130F012C131F0120032C034
:106290002DF033C02EF034C02FF035C030F036C0B2
:1062A00031F012002DC032F02EC033F02FC034F088
:1062B00030C035F031C036F012002DC00EF12EC0C6
:1062C0000FF12FC010F130C011F131C012F11200E6
:1062D00013C12DF014C12EF015C12FF016C130F0EE
:1062E00017C131F0120013C132F014C133F015C1DF
:1062F00034F016C135F017C136F0120018C12DF078
:1063000019C12EF01AC12FF01BC130F01CC131F0A1
:10631000120018C132F019C133F01AC134F01BC198
:1063200035F01CC136F012001DC12DF01EC12EF03B
:106330001FC12FF020C130F021C131F012001DC16A
:1063400032F01EC133F01FC134F020C135F021C13D
:1063500036F0120022C12DF023C12EF024C12FF0FF
:1063600025C130F026C131F0120022C132F023C124
:1063700033F024C134F025C135F026C136F01200C7
:1063800027C12DF028C12EF029C12FF02AC130F0ED
:106390002BC131F0120027C132F028C133F029C1DE
:1063A00034F02AC135F02BC136F0120032C013F19F
:1063B00033C014F134C015F135C016F136C017F1F1
:1063C00012002DC013F12EC014F12FC015F130C0F2
:1063D00016F131C017F112002DC018F12EC019F1BD
:1063E0002FC01AF130C01BF131C01CF112002DC0BA
:1063F0001DF12EC01EF12FC01FF130C020F131C0A1
:1064000021F112002DC022F12EC023F12FC024F162
:1064100030C025F131C026F112002DC027F12EC069
:1064200028F12FC029F130C02AF131C02BF1120020
:106430000EC018F00FC019F010C01AF011C01BF0F8
:1064400012C01CF012000EC01DF00FC01EF010C0D4
:106450001FF011C020F012C021F0120018C00EF081
:1064600019C00FF01AC010F01BC011F01CC012F0C0
:1064700012001D361E361F36203621361200183601
:1064800019361A361B361C361200213220321F32C2
:106490001E321D3212001C321B321A3219321832CF
:1064A000120006D813361436153616361736120073
:1064B0000E360F36103611361236120017321632DB
:1064C0001532143213321200F9DF12321132103247
:1064D0000F320E32120018AE04D019681A681B6809
:1064E0001C68120019AE03D01A681B681C681200E1
:1064F0001AAE02D01B681C6812001BAE01D01C68CB
:1065000012003B923ABE3B828CDE280E0B6ED89076
:106510004BEC32F065EC32F003D80B2EF8D71200BA
:1065200067EC3CF00A0E0A6E00EE0EF0EF50E8B693
:10653000FD0FE8BED00FEE6E0A2EF8D774EC3CF0DB
:1065400012003FD812AE09D0132AD8B4142AD8B4F6
:10655000152AD8B4162AD8B4172A18EC31F035D039
:1065600030D812AE09D0132AD8B4142AD8B4152AB8
:10657000D8B4162AD8B4172A13C00EF014C00FF0DE
:1065800015C010F016C011F017C012F03ABE59EC49
:1065900039F0120016D813C00EF014C00FF015C059
:1065A00010F016C011F017C012F03ABE59EC39F0D5
:1065B000120007D812EC31F008D003D818EC31F0F3
:1065C00004D0F4EC34F0E9EF32F0A6EC33F00AEF4B
:1065D00035F04CD803E111EC31F01AD01AD87F0E07
:1065E000226E2250265E2350275A26C00AF02652D9
:1065F0000FE026BE06D0D89051EC32F00A2EFBD721
:1066000007D00A1E0A2AD89064EC32F00A2EFBD773
:1066100012003A9E2CBE3A8E2C9E11EC31F028C00E
:106620000FF029C010F02AC011F02BC012F02CC0BE
:1066300013F0D89051EC32F065EC32F0128E13C0AA
:1066400026F0136AD89051EC32F01200040E0A6E54
:10665000EE6608D00A2EFCD7EECFE8FF7F0B03E1F1
:10666000D88401D0D89474EC3CF0120067EC3CF074
:1066700000EE28F0EBD767EC3CF000EE2DF0E6D70B
:1066800067EC3CF000EE32F0E1D767EC3CF000EE56
:1066900018F0DCD767EC3CF000EE1DF0D7D767ECC4
:1066A0003CF000EE0EF00A0E0A6EEE66DBD70A2E04
:1066B000FCD7D6D71C6A1BBE1C6835D01B6A1C6A67
:1066C0001AAE31D01B681C682ED01A6A1B6A1C6A6D
:1066D00019AE29D01A681B681C6825D0196A1A6A75
:1066E0001B6A1C6A18AE1FD019681A681B681C68E0
:1066F0001AD011EC31F03A9E1C6A1DD011EC31F029
:106700003A9E1B6A1C6A17D011EC31F03A9E1A6A45
:106710001B6A1C6A10D011EC31F03A9E196A1A6A91
:106720001B6A1C6A08D011EC31F03A9E1CAE03D0F3
:1067300068EC39F03A8E18C013F019C014F01AC082
:1067400015F01BC016F01CC017F000D07F0E266E8F
:10675000000E276E4FEC33F006E1286A296A2A6A98
:106760002B6A2C6A36D010EC34F007E0D89064EC39
:1067700032F0262AD8B4272AF6D713B00AD0D890F8
:1067800051EC32F026062628D8B42706D8B4265273
:10679000F4D70FA00BD00F800F2AD8B4102AD8B48A
:1067A000112AD8B4122AD8B4132ADDD70E6A13904E
:1067B00026C013F064EC32F00FC028F010C029F0AE
:1067C00011C02AF012C02BF013C02CF02C9E3ABE40
:1067D0002C8E1200286A296A2A6A2C6A800E2B6E77
:1067E000F5D7286829682A687F0E2B6E7F0E2C6EDD
:1067F000EDD77F0E186E000E196E2750195C02E15E
:106800002650185CD8B003D0ECDFD88401D0D894DF
:10681000120027AE03D0DEDFD88401D0D894120056
:1068200067EC3CF000EE17F0040E0A6EED660AD03D
:106830000A2EFCD7010EEF6201D002D0EF6602D023
:10684000D88401D0D89474EC3CF012001DC000F143
:106850001EC001F11FC002F120C003F121C004F1EC
:1068600070EC34F00EC007F10FC008F110C009F150
:1068700011C00AF112C00BF100C118F001C119F0EA
:1068800002C11AF003C11BF004C11CF056EC34F035
:1068900007C113F008C114F009C115F00AC116F0C0
:1068A0000BC117F03A9E3BB23A8E1200BADC280EAA
:1068B0000B6ED89005D858EC32F00B2EFAD7120098
:1068C00067EC3CF0050E0A6E00EE18F0D890EF5021
:1068D000E8200700EE6E0A2EFAD774EC3CF01200A6
:1068E00067EC3CF09EDC280E0B6ED8904BEC32F03F
:1068F00065EC32F000EE18F0050E0A6EEFAE02D035
:10690000300EEF5EEFA602D0030EEF5EEE520A2EBF
:10691000F5D70B2EEAD774EC3CF0120002D818EF32
:1069200032F067EC3CF09ADD00EE0EF010EE1DF058
:10693000040E0A6EE650EE5EE650EE5A0A2EFCD7C2
:1069400074EC3CF0120002D818EF32F067EC3CF027
:1069500085DD00EE0EF010EE1DF0E650EE26040E82
:106960000A6EE650EE220A2EFCD774EC3CF01200C0
:1069700000C118F001C119F002C11AF003C11BF0E7
:1069800004C11CF005C122F006C123F0120007C1AA
:106990001DF008C11EF009C11FF00AC120F00BC193
:1069A00021F00CC124F00DC125F012000FC000F140
:1069B00010C001F111C002F112C003F113C004F1C3
:1069C00026C005F127C006F112000FC007F110C064
:1069D00008F111C009F112C00AF113C00BF126C071
:1069E0000CF127C00DF112002DC028F02EC029F0A7
:1069F0002FC02AF030C02BF031C02CF0120032C072
:106A000028F033C029F034C02AF035C02BF036C04E
:106A10002CF0120028C02DF029C02EF02AC02FF033
:106A20002BC030F02CC031F0120028C032F029C049
:106A300033F02AC034F02BC035F02CC036F01200F1
:106A400084EC3CF016E281EC3CF013E23BEC33F0DA
:106A50001AE040EC33F017E099EC3CF004E33BEC37
:106A600033F001E306D09CEC3CF006E340EC33F05D
:106A700003E3C1EC3CF0120099EC3CF003E3B6EC0C
:106A80003CF003D00DD02BEC31F031BE03D036AE4C
:106A900001D0318E31AE03D036BE01D0318E12001E
:106AA0001DD83A9E3ABA3A7E3ABC3A7E15EC39F095
:106AB00012C000F113C001F114C002F115C003F1BE
:106AC00016C004F11ED8A6EC34F018EC32F025EC18
:106AD00031F07F0E1D6E91EC34F01ED03A9A3A9C44
:106AE00031BE3A8A36BE3A8C7FDF09EC33F05EDF86
:106AF00086DF09EC33F069DF10EC31F039DFC7EFE6
:106B000034F010EC31F022C018F023C019F024C08A
:106B10001DF025C01EF012000EC026F00FC027F099
:106B200011EC31F000C10FF001C110F002C111F001
:106B300003C112F004C113F0AAEC33F00AEF35F0F0
:106B400084EC3CF009E281EC3CF006E23BEC33F0F3
:106B500006E140EC33F019E1C1EC3CF012009CEC92
:106B60003CF003E399EC3CF0F7E240EC33F010E149
:106B7000B6EC3CF031BE03D036AE01D0318E31AE32
:106B800003D036BE01D0318E1200CBEC3CF0F2D7F0
:106B9000A5DF3A9E3ABA3A7E3ABC3A7EE3EC39F047
:106BA00005DFAFDF91EC34F018EC32F025EC31F07A
:106BB0007F0E1D6EA6EC34F0AFD740EC33F001E150
:106BC0001200367E00D084EC3CF004E281EC3CF014
:106BD00001E203D0C1EC3CF0120040EC33F001E1E3
:106BE00012003BEC33F003E147EC31F0120017D810
:106BF000A6EC34F022C026F023C027F03A9E12AE55
:106C000003D03A8E59EC39F00EC000F10FC001F1FB
:106C100010C002F111C003F112C004F181D75EDF90
:106C2000FE0E266E000E276E2550235C02E12450D6
:106C3000225C27E013E3242AD8B4252A2750255CB8
:106C400002E12650245C07E125EC31F022C024F05B
:106C500023C025F016D0D89018DCE6D7222AD8B465
:106C6000232A2750235C02E12650225C07E11EEC18
:106C700031F024C022F025C023F003D0D8900BDCE3
:106C8000D3D73ABA68EC39F03ABC77EC39F0120055
:106C900052EC31F020EF35F03BEC33F02DE031BE1B
:106CA0002CD084EC3CF028E25DEC31F0ECD848DFED
:106CB000E1EC31F01E0E0D6E0D4E1ED03CEC31F0AD
:106CC00073EC31F03DDF73EC31F07DDFDCD838DF81
:106CD00073EC31F03650315C0BE13550305C08E13B
:106CE00034502F5C05E133502E5C02E132502D5CB4
:106CF00003E0E1EC31F0E0D71200C1EC3CF012000F
:106D00003BEC33F008E13F0E316E800E306E2D6AA1
:106D10002E6A2F6A120001013F0E266F800E256F2A
:106D2000226B236B246B3F0E216F800E206F1D6B37
:106D30001E6B1F6B0001ECEC31F0E1EC31F022C175
:106D40000EF123C10FF124C110F125C111F126C1AB
:106D500012F11E0E0D6E68EC31F09FEC31F0F0DE9A
:106D600031EC31F0E3EC35F031EC31F03650315CA0
:106D70000BE13550305C08E134502F5C05E13350B5
:106D80002E5C02E132502D5C17E00D4E15D05DEC0B
:106D900031F0AAEC31F06FD816DF02EC32F09FEC44
:106DA00031F04EDEF7EC31F07EEC31F073EC31F087
:106DB00047DEE1EC31F0CFD712003BEC33F008E1D5
:106DC0003F0E316E800E306E2D6A2E6A2F6A1200D1
:106DD0002DC02CF12EC02DF12FC02EF130C02FF17F
:106DE00031C030F1D9EC32F03BD82ADE89DF0DEC2E
:106DF00032F02CC12DF02DC12EF02EC12FF02FC15D
:106E000030F030C131F0E1EC32F03A943ABE3A84DD
:106E100013C00DF027C12DF028C12EF029C12FF08D
:106E20002AC130F02BC131F00D5206E03AA4C5D88A
:106E30003AB4D5D80D2EFAD71200420E366E480E4F
:106E4000356E326A336A346A1200400E366E490E6D
:106E5000356E0F0E346EDA0E336EA20E326E1200E5
:106E6000400E366E130E356E5D0E346E8D0E336E23
:106E7000DE0E326E12003F0E366E800E356E326AB6
:106E8000336A346A1200400E366E326A336A346AEC
:106E9000356A1200410E366E200E356E326A336A44
:106EA000346A1200420E366EC80E356E326A336A8C
:106EB000346A1200440E366E7A0E356E326A336AC8
:106EC000346A1200460E366E1C0E356E400E346E5D
:106ED000326A336A1200470E366EC30E356E500E9C
:106EE000346E326A336A1200490E366E740E356E95
:106EF000240E346E326A336A12004B0E366E180E50
:106F0000356E960E346E800E336E326A12004C0E61
:106F1000366EBE0E356EBC0E346E200E336E326A87
:106F200012004E0E366E6E0E356E6B0E346E280EDF
:106F3000336E326A12003D0E366ECC0E356ECC0EBC
:106F4000346ECC0E336ECD0E326E12003C0E366EA9
:106F5000230E356ED70E346E0A0E336E3D0E326E32
:106F600012003A0E366E830E356E120E346E6E0EB1
:106F7000336E980E326E1200350E366E860E356EFA
:106F8000370E346EBD0E336E060E326E1200300EAA
:106F9000366E890E356E700E346E5F0E336E410E96
:106FA000326E12002B0E366E8C0E356EBC0E346EA9
:106FB000CC0E336E090E326E12006CDF20EF35F00E
:106FC00071DF20EF35F076DF20EF35F07BDF20EF4B
:106FD00035F081DF20EF35F087DF20EF35F05ADF25
:106FE000A0EF35F05FDFA0EF35F064DFA0EF35F004
:106FF00069DFA0EF35F06FDFA0EF35F075DFA0EFB0
:1070000035F03BEC33F003E1C1EC3CF012005DECF9
:1070100031F001013F0E176F800E166F136B146B6A
:10702000156B000128DFDDEC35F0ECEC31F03CECC9
:1070300031F021DFE3EC35F0F7EC31F07EEC31F0AC
:107040009FEC31F0A0EC35F0ECEC31F002EC32F0DA
:107050005DEC31F0280E0D6E68EC31F014DFE3ECDE
:1070600035F0E1EC31F07EEC31F0B5EC31F020ECB4
:1070700035F0B5EC31F020EC35F0ECEC31F073ECA0
:1070800031F0A0EC35F031EC31F0E3EC35F031ECDF
:1070900031F03650315C0BE13550305C08E1345052
:1070A0002F5C05E133502E5C02E132502D5C05E08F
:1070B0000D4E03D05DEC31F0CFD7E5DE20EF35F09B
:1070C0000101276B00014AEC37F048D806E3EFECEA
:1070D00037F00101272B0001F6D793DFC1DEA0ECCA
:1070E00035F010EC31F027C113F0135206E0A6EC96
:1070F00033F015EC35F0E3EC35F012007ED81CAE21
:1071000014D021AE29D05AD81C50215C0BE11B5061
:10711000205C08E11A501F5C05E119501E5C02E179
:1071200018501D5CD8B016D017D01CBE02D021BE9E
:1071300011D044D81C50215C0BE11B50205C08E1AD
:107140001A501F5C05E119501E5C02E118501D5CCD
:10715000D8B002D0D89001D0D88012004ED81CAE42
:1071600014D021AE29D02AD81C50215C0BE11B5031
:10717000205C08E11A501F5C05E119501E5C02E119
:1071800018501D5CD8B016D017D01CBE02D021BE3E
:1071900011D014D81C50215C0BE11B50205C08E17D
:1071A0001A501F5C05E119501E5C02E118501D5C6D
:1071B000D8B002D0D88001D0D89012003BEC33F088
:1071C00003E11EEC31F00FD0D8903FEC32F0D890B4
:1071D0001B321A32193218321B8E40EC33F003E1A5
:1071E00025EC31F009D0D89039EC32F0D89020322B
:1071F0001F321E321D32208E12002DC018F02EC0FC
:1072000019F02FC01AF030C01BF031C01CF032C092
:107210001DF033C01EF034C01FF035C020F036C062
:1072200021F0120002D818EF32F067EC3CF037D8AA
:10723000050E0A6E00EE1DF020EE0EF011EC31F09E
:1072400010EE18F0050E0B6E0AC00CF00B500C2659
:107250000C060C06EF50E602F350DE26D9CF37F0CD
:10726000DACF38F0F450DE22E86ADE220C2EFCD7AA
:1072700037C0D9FF38C0DAFF0B2EE6D7EE5220EE2A
:107280000EF0060E0C6E0A500C5EDE520C2EFDD770
:107290000A2ED6D774EC3CF03AB20BD812003A92D0
:1072A0001CAE02D015D83A7221AE02D020D83A7264
:1072B00012000E1E0F1E101E111E121E0E2AD8B412
:1072C0000F2AD8B4102AD8B4112AD8B4122A12001E
:1072D000181E191E1A1E1B1E1C1E182AD8B4192A85
:1072E000D8B41A2AD8B41B2AD8B41C2A12001D1EDE
:1072F0001E1E1F1E201E211E1D2AD8B41E2AD8B4F1
:107300001F2AD8B4202AD8B4212A1200C8DF67EC7B
:107310003CF011EC31F0050E0A6E00EE1DF0EE6649
:1073200005D00A2EFCD774EC3CF012000A6A0A2A37
:10733000D89021BE1CD01D361E361F362036213671
:1073400021501C5C0BE120501B5C08E11F501A5CB3
:1073500005E11E50195C02E11D50185CE8E211ECD9
:1073600031F0D890213220321F321E321D3221508E
:107370001C5C0BE120501B5C08E11F501A5C05E10E
:107380001E50195C02E11D50185C0AE31D50185E86
:107390001E50195A1F501A5A20501B5A21501C5A5D
:1073A00058EC32F00A2EDDD777DF18C01DF019C077
:1073B0001EF01AC01FF01BC020F01CC021F018ECFA
:1073C00032F074EF3CF0290E0A6E11EC31F02150CE
:1073D0001C5C0BE120501B5C08E11F501A5C05E1AE
:1073E0001E50195C02E11D50185C0BE31D50185E25
:1073F0001E50195A1F501A5A20501B5A21501C5AFD
:10740000D88051EC32F0D8903FEC32F021501C5C27
:107410000BE120501B5C08E11F501A5C05E11E5077
:10742000195C02E11D50185C0BE31D50185E1E50E4
:10743000195A1F501A5A20501B5A21501C5AD880D2
:107440000A2EDFD7120067EC3CF03A921CAE02D055
:107450003FDF3A8211EC31F0280E0A6E0A0E0B6EF5
:1074600000EE0EF0EF500F0B0C6E050E0C5CD8A06A
:1074700002D0030EEF26EF50F00B0C6E500E0C5C9A
:10748000D8A002D0300EEF26EC520B2EEBD7D890BE
:107490003FEC32F051EC32F00A2EE0D774EC3CF0C5
:1074A000120084EC3CF015E29CEC3CF01CE22FD87E
:1074B00044D85AD83B941200030E376409D038667A
:1074C000372A3AB4372A030E375E375035EC24F0AA
:1074D0001200F2DF000EF86E610EF76EDC0EF66E33
:1074E00046EC24F01200E8DF000EF86E610EF76E35
:1074F000E00EF66E46EC24F0120084EC3CF0E9E27B
:107500009CEC3CF0F0E203D82FD83B94120067ECDF
:107510003CF000EE17F011EE31F00A0E0C6EEDCFDC
:107520000AF00A380B6E56D80AC00BF053D80C2E4E
:10753000F6D7E76A74EC3CF0120067EC3CF0385286
:1075400010E001EE44F011EE44F0140E0A6E38C063
:107550000BF0E5500A060B2EFCD7E5CFEDFF0A2E07
:10756000FCD774EC3CF0120067EC3CF00A0E0B6E9A
:1075700038500B2637500B5CD8B002D00BC037F018
:107580003750385CD8A003D038C037F0372A38508D
:10759000375E3706090E0A6E37500A5E01EE31F08B
:1075A0000A5204E0EECFE8FF0A2EFCD73AA405D039
:1075B0002B0E3ABE2D0E29EC3BF03A8019D83A90AA
:1075C00013D8385204E02C0E29EC3BF009D874ECA7
:1075D0003CF012000B500F0B3009E8CFE6FF120011
:1075E00038C00CF03B9606D0010E0C6E3B9602D0D4
:1075F00037C00CF00C5226E03AA006D0EFCF0AF0CC
:10760000300E0A5CD8A43A903BA611D00CC018F0FA
:10761000020E186202D023EC3BF0050E186202D075
:1076200023EC3BF0080E186202D023EC3BF0EECFC7
:10763000E8FF3AB003D029EC3BF002D025EC3BF058
:107640000C2EDAD71200200E04D0200E3BB4300EE0
:1076500000D0086E3C6603D008508BEC23F0010E7E
:107660003C6203D00850E6EC17F0020E3C6203D0F7
:10767000085052EC24F0120067EC3CF00A0E0A6E3F
:1076800038500A5E00EE0EF0EF500A4E0CD0EF506C
:107690000A4E02D0EE52F8D7EE52186E490E186418
:1076A00009D0010E06D00F0B186E040E186402D01C
:1076B000100EEF260A0E0A6E00EE0EF0EF500700D5
:1076C000EE6EE86AEF220A2EF9D774EC3CF0120055
:1076D00067EC3CF0050E0A6E0A0E0B6E00EE17F01A
:1076E000EDCF18F01850F00B07E10B0618500F0BF8
:1076F00003E10B060A2EF4D70BC018F00B5074EC04
:107700003CF01200CBEC3CF011EC31F023EC3AF001
:107710000EC013F00FC014F010C015F011C016F019
:1077200012C017F0050E376E386A3A943B943A98B7
:107730003B963C6A120084EC3CF045E29CEC3CF049
:1077400042E2F4EC34F0E9EC32F00EC000F10FC08C
:1077500001F110C002F111C003F112C004F113C015
:1077600018F014C019F015C01AF016C01BF017C09D
:107770001CF023EC3AF00EC007F10FC008F110C066
:1077800009F111C00AF112C00BF100C118F001C1DA
:1077900019F002C11AF003C11BF004C11CF081EC06
:1077A00032F007C113F008C114F009C115F00AC185
:1077B00016F00BC117F0140E376E0A0E386E3A9899
:1077C0003B963B943C6A3A9412005DEC31F0396A86
:1077D000319E3BEC33F014E04AEC37F0AEEC38F07D
:1077E00001E004E3EFEC37F0392AF6D73BEC37F051
:1077F0007EEC38F005E004E3DDEC37F03906F6D72F
:107800009BEC3BF03CEC31F031BE3A8E0B0E376E08
:107810000A0E386E3A843A983C6A12007DEC3AF0CF
:10782000650E29EC3BF03A9E39BE3A8E39BE396C72
:107830001EEC31F039C018F082EC3BF03A8448DF9E
:1078400018C037F07DEC3AF0120068EC31F031EC02
:1078500031F0DDEC35F00DEC32F094EC31F089ECE8
:1078600031F0DDEC35F052EC31F027C12DF028C1BC
:107870002EF029C12FF02AC130F02BC131F0A0EC3D
:1078800035F00DEC32F0AAEC31F089EC31F0DDECA2
:1078900035F0CBEC31F020EC35F031EC31F0E3ECAD
:1078A00035F0120067EC3CF01EEC31F0050E0A6E6C
:1078B00010EE0EF020EE18F0E6500F0BDF6EE638FB
:1078C000F00BDE120A2EF8D774EC3CF01200E9CF70
:1078D00045F1EACF46F1E1CF47F1E2CF48F1D9CF08
:1078E00049F1DACF4AF1120045C1E9FF46C1EAFF8A
:1078F00047C1E1FF48C1E2FF49C1D9FF4AC1DAFFF0
:107900001200FFEC34F003D0F4EC34F000D02C9EE5
:107910007F0E2C620CD0800E2B6207D02A6605D019
:10792000296603D0286601D002D0D88001D0D89033
:107930001200FFEC34F003D0F4EC34F000D02C9EB5
:107940007F0E2C620BD0800E2B6208D02A6606D0E8
:10795000296604D0286602D0D88001D0D8901200C1
:1079600002D80AEF35F005D82C8E120002D80AEFA3
:1079700035F07F0E2C6E800E2B6E286A296A2A6ADB
:10798000120002D80AEF35F07F0E2C6E28682968A5
:107990002A682B68120002D80AEF35F0286A296A93
:1079A0002A6A2B6A2C6A1200410E366EA00E356EC2
:1079B000326A336A346A1200D4EC3CF0A0EC35F041
:1079C000DDEC36F05DEC31F03BEC37F0E3EC35F01C
:1079D000E1EC31F03CEC31F03BEC37F0DDEC35F034
:1079E00052EC31F068EC31F0A0EC35F012004BC1F4
:1079F0002DF04CC12EF04DC12FF04EC130F04FC1D3
:107A000031F0EFEC37F0DDEC36F02DC055F12EC043
:107A100056F12FC057F130C058F131C059F1120062
:107A200055C12DF056C12EF057C12FF058C130F07E
:107A300059C131F0F5EC37F01DEC37F020EC35F0A2
:107A40004CEC36F02DC060F12EC061F12FC062F118
:107A500030C063F131C064F1120060C12DF061C12A
:107A60002EF062C12FF063C130F064C131F001012A
:107A7000010E656F0001BCEC37F07EEC38F009E3D5
:107A80000101040E656F0001ECEC37F0E3EC37F018
:107A900018D0B1EC37F07EEC38F007E30101030EAB
:107AA000656F0001ECEC37F00CD03BEC37F07EEC6E
:107AB00038F007E30101020E656F0001E3EC37F0D7
:107AC00000D02DC05BF12EC05CF12FC05DF130C045
:107AD0005EF131C05FF1120055C12DF056C12EF09C
:107AE00057C12FF058C130F059C131F00101030ED8
:107AF0005A6F0001D2EC37F07EEC38F00BE3ECEC7F
:107B000037F0ECEC37F0E3EC37F00101080E5A6F78
:107B100000014CD0C7EC37F07EEC38F009E3ECEC18
:107B200037F0ECEC37F00101070E5A6F00013ED040
:107B3000BCEC37F07EEC38F009E3ECEC37F0E3EC2A
:107B400037F00101060E5A6F000130D0B1EC37F06A
:107B50007EEC38F007E3ECEC37F00101050E5A6FCC
:107B6000000124D03BEC37F07EEC38F007E3E3EC87
:107B700037F00101040E5A6F000118D074EC37F091
:107B8000AEEC38F007E3FEEC37F00101010E5A6F5E
:107B900000010CD05AEC37F0AEEC38F007E3F5EC0E
:107BA00037F00101020E5A6F000100D02DC050F1D4
:107BB0002EC051F12FC052F130C053F131C054F1F9
:107BC000120050C12DF051C12EF052C12FF053C1FF
:107BD00030F054C131F09BEC3BF0050E376E010ED6
:107BE000386E4AEC37F07EEC38F003E3040E386E62
:107BF0000FD052EC37F07EEC38F003E3030E386E12
:107C000007D05AEC37F07EEC38F002E3020E386E03
:107C100067D83CEC3BF07DEC3AF05AC118F0030E0B
:107C2000186209D0000EF86E610EF76EE40EF66E63
:107C300046EC24F054D0040E186209D0000EF86E01
:107C4000610EF76EE80EF66E46EC24F048D0050E95
:107C5000186209D0000EF86E610EF76EEC0EF66E2B
:107C600046EC24F03CD0060E186209D0000EF86EE7
:107C7000610EF76EF00EF66E46EC24F030D0070E73
:107C8000186209D0000EF86E610EF76EF40EF66EF3
:107C900046EC24F024D0020E186209D0000EF86ED3
:107CA000610EF76EFC0EF66E46EC24F018D0010E55
:107CB000186209D0000EF86E620EF76E000EF66EB6
:107CC00046EC24F00CD0080E186209D0000EF86EB5
:107CD000610EF76EF80EF66E46EC24F000D012003E
:107CE00068EC3BF0030E186402D0010E386E030EF0
:107CF000186202D0020E386E020E186202D0030E15
:107D0000386E010E186202D0040E386E000E186232
:107D100002D0040E386E12005BC12DF05CC12EF053
:107D20005DC12FF05EC130F05FC131F09BEC3BF0E4
:107D3000060E376E010E386E5AEC37F07EEC38F0D6
:107D400002E3020E386E52EC37F07EEC38F002E3BC
:107D5000030E386E4AEC37F07EEC38F002E3040E86
:107D6000386EBEDF3CEC3BF07DEC3AF065C118F0BC
:107D7000010E186209D0000EF86E620EF76E040E46
:107D8000F66E46EC24F024D0020E186209D0000EE4
:107D9000F86E620EF76E080EF66E46EC24F018D000
:107DA000030E186209D0000EF86E620EF76E0C0E0C
:107DB000F66E46EC24F00CD0040E186209D0000ECA
:107DC000F86E620EF76E100EF66E46EC24F000D0E0
:107DD00012004BC12DF04CC12EF04DC12FF04EC101
:107DE00030F04FC131F09BEC3BF0050E376E020EC8
:107DF000386E3CEC3BF068EC3BF0030E186004D0AE
:107E0000040E376E020E386E020E186404D0040E93
:107E1000376E010E386E24D04BC12DF04CC12EF0C0
:107E20004DC12FF04EC130F04FC131F09BEC3BF013
:107E3000040E376E010E386E3CEC3BF068EC3BF004
:107E4000030E186004D0030E376E010E386E020E5A
:107E5000186406D0040E376E000E386E3CEC3BF012
:107E60003A847DEC3AF0000EF86E620EF76E140E56
:107E7000F66E46EC24F0120050C12DF051C12EF0E8
:107E800052C12FF053C130F054C131F09BEC3BF0A4
:107E9000040E376E010E386E4AEC37F07EEC38F087
:107EA00003E3030E386E0FD052EC37F07EEC38F05F
:107EB00003E3020E386E07D05AEC37F07EEC38F050
:107EC00002E3010E386E3CEC3BF065D87DEC3AF0F5
:107ED0005AC118F0030E186209D0000EF86E610E38
:107EE000F76EE40EF66E46EC24F054D0040E1862E1
:107EF00009D0000EF86E610EF76EE80EF66E46ECD5
:107F000024F048D0050E186209D0000EF86E610EFC
:107F1000F76EEC0EF66E46EC24F03CD0060E1862BE
:107F200009D0000EF86E610EF76EF00EF66E46EC9C
:107F300024F030D0070E186209D0000EF86E610EE2
:107F4000F76EF40EF66E46EC24F024D0020E1862A2
:107F500009D0000EF86E610EF76EFC0EF66E46EC60
:107F600024F018D0010E186209D0000EF86E620ECF
:107F7000F76E000EF66E46EC24F00CD0080E186278
:107F800009D0000EF86E610EF76EF80EF66E46EC34
:107F900024F000D0120068EC3BF0030E186404D00B
:107FA000050E376E000E386E030E186202D0010EF9
:107FB000386E020E186202D0020E386E010E186280
:107FC00002D0030E386E000E186202D0030E386E17
:107FD000120050C12DF051C12EF052C12FF053C1EB
:107FE00030F054C131F09BEC3BF0030E376E010EC4
:107FF000386E4AEC37F07EEC38F003E3020E386E50
:1080000011D052EC37F07EEC38F003E3010E386EFD
:1080100009D05AEC37F07EEC38F004E3000E386EED
:10802000040E376E3CEC3BF065D87DEC3AF05AC15B
:1080300018F0030E186209D0000EF86E610EF76E8C
:10804000E40EF66E46EC24F054D0040E186209D00B
:10805000000EF86E610EF76EE80EF66E46EC24F038
:1080600048D0050E186209D0000EF86E610EF76E4A
:10807000EC0EF66E46EC24F03CD0060E186209D0E9
:10808000000EF86E610EF76EF00EF66E46EC24F000
:1080900030D0070E186209D0000EF86E610EF76E30
:1080A000F40EF66E46EC24F024D0020E186209D0CD
:1080B000000EF86E610EF76EFC0EF66E46EC24F0C4
:1080C00018D0010E186209D0000EF86E620EF76E1D
:1080D000000EF66E46EC24F00CD0080E186209D0A3
:1080E000000EF86E610EF76EF80EF66E46EC24F098
:1080F00000D0120068EC3BF0030E186404D0040EAC
:10810000376E000E386E030E186204D0040E376E00
:10811000000E386E020E186202D0010E386E010E8B
:10812000186202D0020E386E000E186202D0020EE3
:10813000386E120050C12DF051C12EF052C12FF0F7
:1081400053C130F054C131F09BEC3BF0030E376E5D
:10815000010E386E4AEC37F07EEC38F003E3020E85
:10816000386E11D052EC37F07EEC38F003E3010E9C
:10817000386E09D05AEC37F07EEC38F004E3000E8C
:10818000386E040E376E3CEC3BF0B4DF020E3C6EF2
:108190007DEC3AF012005AC118F0030E186209D0B3
:1081A000000EF86E610EF76EE40EF66E4CEC24F0E5
:1081B00054D0040E186209D0000EF86E610EF76EEE
:1081C000E80EF66E4CEC24F048D0050E186209D08B
:1081D000000EF86E610EF76EEC0EF66E4CEC24F0AD
:1081E0003CD0060E186209D0000EF86E610EF76ED4
:1081F000F00EF66E4CEC24F030D0070E186209D069
:10820000000EF86E610EF76EF40EF66E4CEC24F074
:1082100024D0020E186209D0000EF86E610EF76EBF
:10822000FC0EF66E4CEC24F018D0010E186209D04A
:10823000000EF86E620EF76E000EF66E4CEC24F037
:108240000CD0080E186209D0000EF86E610EF76EA1
:10825000F80EF66E4CEC24F000D01200986E1283EB
:108260003C00000086C2986E12833C00000086C26B
:108270000C022BD041040002000000E0400FC800B7
:10828000640630751E320609080A0B0A0D021E002C
:108290000609080A0B0A0E021E000609080A0B0A44
:1082A0000F020F000609080A0B0A0F021400060944
:1082B000080A0B0A0F021E000609080A0B0A0F0221
:1082C00028000609080A0B0A0F0232000609080AEC
:1082D0000B0A100232000609080A0B0A11023200CA
:1082E0000609080A0B0A1202320003000401050203
:1082F0000F021E000306040705080D0232010306E3
:10830000040705080D0232050306040705080D02DF
:10831000323D0609080A0B0A0F0232000609080A54
:108320000B0A0F0232000609080A0B0A0F0232007C
:108330000609080A0B0A0F0232000609080A0B0A8E
:0E8340000F0232000609080A0B0A0F02320073
:020000040030CA
:0300010028192398
:02000500BD80BC
:0200000400F00A
:10000000986E12833C00000086C2986E12833C00FA
:10001000000086C20C022BD041040002000000E068
:10002000400FC800640630751E320609080A0B0A24
:100030000D021E000609080A0B0A0E021E00060920
:10004000080A0B0A0F020F000609080A0B0A0F0222
:1000500014000609080A0B0A0F021E000609080A06
:100060000B0A0F0228000609080A0B0A0F023200C9
:100070000609080A0B0A100232000609080A0B0AD0
:10008000110232000609080A0B0A120232000300AC
:10009000040105020F021E000306040705080D02F5
:1000A00032010306040705080D02320503060407A2
:1000B00005080D02323D0609080A0B0A0F0232003C
:1000C0000609080A0B0A0F0232000609080A0B0A81
:1000D0000F0232000609080A0B0A0F023200060955
:1000E000080A0B0A0F0232000609080A0B0A0F025F
:0200F0003200DC
:00000001FF
